:020000040800F2
:105000007897002019FE000845FF000849FF0008B6
:105010004DFF000851FF000855FF00080000000088
:105020000000000000000000000000008FE1000808
:105030005DFF00080000000049E1000835BA0008E3
:1050400069FF00086DFF000871FF000875FF000888
:1050500079FF0008DDE2000881FF000885FF0008F5
:1050600089FF00088DFF000891FF000895FF0008E8
:10507000B17600089DFF000831510008A5FF000827
:10508000A9FF000881510008B1FF0008B5FF000822
:10509000B9FF0008BDFF0008C1FF0008C5FF0008F8
:1050A000C9FF0008CDFF0008D1FF0008D5FF0008A8
:1050B000D9FF0008DDFF0008E1FF0008E5FF000858
:1050C000E9FF0008EDFF0008F1FF0008F5FF000808
:1050D000F9FF000865510008B55100080177000884
:1050E000090001080D000108110001081500010860
:1050F000190001081D000108210001082500010810
:10510000290001082D0001083100010835000108BF
:1051100005520008915200084100010845000108AD
:10512000490001084D00010851000108D151000853
:1051300080B54FF4005001F0B2FE002807D04FF4C4
:10514000005001F0C1FEDFF8000A00F03BF94FF417
:10515000004001F0A4FE002803D04FF4004001F00D
:10516000B3FE01BD80B540F22551DFF8E00901F042
:1051700097FF002803D0DFF8D00900F0E4F801BD64
:1051800080B55FF0007001F08AFE002807D05FF064
:10519000007001F099FEDFF8B80900F013F95FF034
:1051A000006001F07CFE002803D05FF0006001F099
:1051B0008BFE01BD80B540F22551DFF8980901F062
:1051C0006FFF002803D0DFF8880900F0BCF801BDAC
:1051D00080B5DFF8840901F062FE002807D0DFF80F
:1051E000780901F071FEDFF8740900F0EBF8DFF8E0
:1051F000C40D01F054FE002803D0DFF8B80D01F013
:1052000063FE01BD80B540F22551DFF8540901F07D
:1052100047FF002803D0DFF8440900F094F801BDEF
:1052200038B504000D002A0092B22100DFF8CC0D41
:1052300001F07AFC31BD38B504000D000421DFF81F
:10524000C00D02F019F801280ED100F003FBDFF8C1
:10525000140902F096F80421DFF8A40D02F01CF8FE
:105260004FF4FA7002F084FC02F062FD64210091B8
:10527000002302000221DFF8100D006803F035FA68
:105280002A0092B22100DFF8C80801F04DFC31BDC0
:1052900080B540F22661DFF8200D01F001FF002803
:1052A0002AD0DFF8180D0088DFF8141D098888421D
:1052B0000FD3002240F22661DFF8FC0C01F0ACFEB7
:1052C0000020DFF8F81C08800020DFF8301D086699
:1052D0001EE0DFF8300DDFF8E41C0988095C89B2B4
:1052E000DFF8D40C01F0CEFEDFF8D00C0088401CB3
:1052F000DFF8C81C08800BE040F22551DFF8B80C3D
:1053000001F0CEFE002803D0DFF8F00C00F01BF80F
:1053100001BD38B504000D002A0092B22100DFF86B
:10532000280801F001FC31BD10B50400DFF81808B1
:10533000C4604FF48060DFF810188882DFF8080836
:1053400000F094FE10BD38B5040000200090B4F8C1
:105350005800FF2802DB0020A4F85800B4F8585089
:10536000681CA4F85800A06801F090FE216DADB251
:10537000685402F0DDFCC01DE065B4F85800012857
:105380001FD1206D0078682803D0206D0078EB28AD
:1053900012D100A9DFF8D00C006803F0ACFD009832
:1053A00000280ED05FF08050DFF8D81D0860BFF3F2
:1053B0004F8FBFF36F8F04E00020A4F85800002047
:1053C000E06531BD10B5040000202066A068DFF85C
:1053D0008417884204D0A068DFF8841788420BD174
:1053E000A068808950F00400A1688881012240F201
:1053F0002551A06801F010FE10BD38B504000D0065
:10540000EDB22A0092B22100DFF87C0D006D04F0AD
:1054100043F8EDB2DFF8700DA0F85A50DFF86C0DCC
:1054200001F0AFFFEDB2290089B2DFF85C0D006D2D
:1054300002F04CF8002300220021DFF84C0D4068F8
:1054400003F0F3FB31BD2DE9F04104000D0026000F
:10545000701C04F057F80700A046042216F10A0158
:1054600015F10D0004F018F8002080B2042808DAC5
:1054700080B24119497B333980B242195173401CC3
:10548000F3E7707A0C2830D10422DFF8041D15F1FF
:105490000D0004F025F9002808D10422DFF8F41CDF
:1054A00015F10D0004F01CF9002851D00020717A8C
:1054B00080B289B2884208D280B28119897A3339A0
:1054C00080B282199172401CF1E7FFB2002F3FD0E9
:1054D0000020287098F80E006870072218F10F015C
:1054E000A81D03F0D9FF012033E0707A06282FD1E0
:1054F0000222DFF8A41C15F10D0004F0F1F80028D9
:1055000008D10222DFF8901C15F10D0004F0E8F834
:1055100000281DD00020717A80B289B2884208D25A
:1055200080B28119897A333980B282199172401C14
:10553000F1E70120287010206870062218F101019F
:10554000A81D03F0A9FF98F80C002873012000E0C3
:105550000020BDE8F08138B50400250068202870DF
:10556000681C04F01AF86820E8719320287206205D
:10557000687215F10A0004F010F80020697AC0B2D0
:10558000884208D2C0B24119897A3331C0B2421977
:105590009172401CF2E71021280004F08FF8287463
:1055A0001620687412222900DFF89C0501F0BCFA6D
:1055B000DFF8E80B01F0E5FE1221280001F086FF7C
:1055C00031BD38B50400250068202870A02068701F
:1055D000A120A870A220E870A3202871A4206871DF
:1055E000A520A8716820E8719F20287208206872A1
:1055F000AF20A8720220E8720622FF2115F10C00EC
:1056000003F05AFF0020697AC0B2884208D2C0B2C3
:105610004119897A3331C0B242199172401CF2E7C4
:105620001221280004F04AF8A8741620E874142205
:105630002900DFF8140501F077FADFF8600B01F0BC
:10564000A0FE1421280001F041FF31BD10B5040077
:10565000A4B2200001280CD002280AD0032825D0AB
:1056600004283ED005283CD0072857D0082863D00E
:1056700071E04FF41660DFF8D814C8604FF4806012
:10568000DFF8CC1488824FF41660DFF8D014C860BD
:105690004FF48060DFF8C4148882DFF8C00400F0A3
:1056A000E5FCDFF8AC0400F0E1FC54E04FF41660D8
:1056B000DFF89C14C8600020DFF8941488824FF44F
:1056C0001660DFF89814C8600020DFF89014888214
:1056D000DFF8880400F0CAFCDFF8740400F0C6FCB0
:1056E00039E04FF49660DFF86814C8604FF48060CA
:1056F000DFF85C1488824FF49660DFF86014C860AD
:105700004FF48060DFF854148882DFF8500400F012
:10571000ADFCDFF83C0400F0A9FC1CE04FF49660FF
:10572000DFF8D818C8600020DFF8D0188882DFF8CA
:10573000CC0800F09BFC0EE04FF41660DFF8BC18BC
:10574000C8604FF48060DFF8B4188882DFF8AC08D6
:1057500000F08CFCFFE710BDF8B504000D0016004A
:105760001F00DFF8DC0D0088A4B2A04203D02000A7
:1057700080B2FFF76BFFA4B2200001280ED00228F0
:1057800013D0032818D004281CD0052820D00728BF
:1057900024D0082828D00A282CD031E03B00320041
:1057A0000121280004F095F931E03B00320000218E
:1057B000280004F08EF92AE03A003100280004F0B5
:1057C000C7F924E03A003100280004F06AFA1EE02C
:1057D0003A003100280004F087FA18E03A0031005E
:1057E000280004F038FA12E03A003100280004F0F2
:1057F000FDF90CE03A003100280004F094FA06E0CC
:10580000DFF83C0D048000203880002003E0DFF842
:10581000300D04800120F2BD10B40200002080B2DF
:1058200089B288420CD289B28B1C80B21B1A89B211
:1058300080B20C1AA41814F8014C9C54401CEEE7DA
:10584000FE201070FE205070FE209070C81C80B2A8
:1058500010BC704780B50121142004F080FC0420A6
:10586000ADF8000010208DF8030003208DF8020031
:1058700000A9DFF88C0701F057FC0421DFF880074E
:1058800001F007FD01BD10B504000421DFF8700729
:1058900001F0FFFCDFF8AC0C01F073FD10BD70B53A
:1058A00004000D002E0068203070701C03F075FE9F
:1058B0006820F071912030723D207072042214F142
:1058C0000D0116F10A0003F0E7FD0522EE2116F1A5
:1058D0000E0003F0F1FD6078F074052214F111015F
:1058E00016F1140003F0D8FD2C207076042200215C
:1058F00016F11A0003F0E0FD0222EE2116F11E005F
:1059000003F0DAFD0322EE2116F1200003F0D4FDAE
:105910001022EE2116F1230003F0CEFD0322EE212A
:1059200016F1330003F0C8FD0722002116F13600FE
:1059300003F0C2FD022214F1150116F13D0003F03F
:10594000ABFD607886F83F000722A11D16F14000EC
:1059500003F0A2FD0020717AC0B2884208D2C0B222
:105960008119897A3331C0B282199172401CF2E7F1
:105970004721300003F0A2FE86F84700162086F883
:10598000480070BD70B504000D002E006820307016
:10599000701C03F002FE6820F071912030724020EC
:1059A0007072042214F10D0116F10A0003F074FD67
:1059B0000322EE2116F10E0003F07EFD0522EE21FA
:1059C00016F1110003F078FD6078B075052214F12E
:1059D000110116F1170003F05FFD2C20307704222F
:1059E000002116F11D0003F067FD1522EE2116F1CE
:1059F000210003F061FD0322EE2116F1360003F0D1
:105A00005BFD0722EE2116F1390003F055FD02225D
:105A100014F1150116F1400003F03EFD607886F8A0
:105A200042000722A11D16F1430003F035FD0020BE
:105A3000717AC0B2884208D2C0B28119897A3331F2
:105A4000C0B282199172401CF2E74A21300003F083
:105A500035FE86F84A00162086F84B0070BD70B5FA
:105A600004000D002E00682030700622A11D701C5D
:105A700003F012FD6820F0719120307217207072CF
:105A8000022214F10D0116F10A0003F005FD0020B9
:105A9000307310207073052214F1110116F10E00FD
:105AA00003F0FAFC0422002116F1130003F004FDB8
:105AB0002C20F0750722002116F1180003F0FCFCE1
:105AC000022214F1150116F11F0003F0E5FC00207D
:105AD000717AC0B2884208D2C0B28119897A333152
:105AE000C0B282199172401CF2E72121300003F00C
:105AF000E5FD86F82100162086F8220070BD38B535
:105B000004000D002078002803D0022819D013D3F8
:105B100018E00422DFF8781614F10D0003F0E0FD20
:105B2000002804D029002000FFF7B9FE03E0290077
:105B30002000FFF727FF05E029002000FFF78FFF77
:105B400000E0FFE731BD0000F00200200038014016
:105B5000540300200044004000000210B80300205D
:105B6000004C004078FD00082DE9F84304000D00CA
:105B700016001F00DDF82080A4B2200001280CD000
:105B800002280AD0032816D0042822D005282ED0B7
:105B900007283AD0082846D053E017F115000090A6
:105BA00017F11103BA1DF6B2310089B2280004F0D2
:105BB000BBF8814647E017F11500009017F111037B
:105BC000BA1DF6B2310089B2280004F0F6F8814619
:105BD00039E017F11500009017F11103BA1DF6B264
:105BE000310089B2280004F0A9F981462BE017F1B1
:105BF0001500009017F11103BA1DF6B2310089B2F9
:105C0000280004F0C6F981461DE017F11500009048
:105C100017F11103BA1DF6B2310089B2280004F061
:105C200046F981460FE017F11500009017F11103B6
:105C3000BA1DF6B2310089B2280004F000F981469D
:105C400001E0002081465FFA89F9B9F1000F06D022
:105C5000B8F1000F03D041463800FFF750FF484627
:105C6000C0B2BDE8F28370B504000D001600002D2F
:105C700028D0708868713079A8717079E871E4B2C1
:105C8000002C04D0287C012801D001202874E4B223
:105C9000002C01D0002001E0E87B401CE873E87B89
:105CA000032801DB02202874052216F1110115F1E9
:105CB000110003F0F1FB022216F1150115F1160097
:105CC00003F0EAFB70BD2DE9F04F83B004000D0036
:105CD000160006275FF009085FF00C094FF47A7A86
:105CE000E4B2002C06D101200700072080460A20DC
:105CF00081461DE0E4B2062C02DAE4B2270017E088
:105D0000E4B2062C01D100203BE1E4B2092C02DA16
:105D1000E4B227000CE0E4B2092C01D1002030E10C
:105D2000E4B20C2C02DAE4B2A14601E0002028E142
:105D30004FF47A708246BFB2062F1FDA01ABDFF84C
:105D4000902CA91D380080B2FFF706FDBDF80410A5
:105D5000DFF87C0CFFF760FDADF80400BDF804101F
:105D6000DFF86C0CFFF767FADFF8680C01F009FB4D
:105D7000BDF80410DFF8580C01F0A8FB1FFA88F8F2
:105D8000B8F1090F2BDA1FFA88F8B8F1080F06D11D
:105D900040F6C410824502D240F6C410824601ABE0
:105DA000DFF8342CA91D404680B2FFF7D5FCBDF8C2
:105DB0000410DFF8240CFFF72FFDADF80400BDF848
:105DC0000410DFF8140CFFF72BFADFF8100C01F0C9
:105DD000D8FABDF80410DFF8000C01F077FB1FFAC9
:105DE00089F9B9F10C0F0FDA1FFA89F9B9F10A0F25
:105DF00006D141F28830824502D241F28830824693
:105E0000DFF8DC0B01F0BDFA002302220021DFF8ED
:105E1000D40B006802F01EFB4FF4FA7000FB0AF08E
:105E20004FF47A71B0FBF1F1DFF8BC0B006803F0BE
:105E3000E9FA8346BBF1000F12D001F079FF64212B
:105E400000910023020002214F48006802F04DFC3F
:105E5000002302220021DFF8940B006802F0FAFA16
:105E6000DFF8B8054068834523D1002300220021D4
:105E7000DFF8A805406803F0B3F8002028716F80B0
:105E800001F056FF020064200090002302213E48EA
:105E9000006802F02AFC00962B00DFF88005B0F8BD
:105EA0005A20D2B2DFF87405016D6888FFF75CFEF6
:105EB00067E052484068834521D100230022002139
:105EC0004E48406803F08CF803202871A5F8028042
:105ED00001F02EFF642100910023020002212A48D4
:105EE000006802F002FC00962B004448B0F85A20EB
:105EF000D2B24248016D6888FFF736FE41E0E4B255
:105F0000002C0CD001F014FF64210091002302004A
:105F100002211D48006802F0E8FB002031E01FFA72
:105F200088F8B8F1090F02DA18F1010801E05FF012
:105F30000908BFB2062F01DA7F1C00E006271FFA0E
:105F400089F9B9F10C0F02DA19F1010901E05FF0EA
:105F50000C09BFB21FFA88F818EB07001FFA89F97D
:105F600019EB00001B28FFF6E3AE01F0E1FE64210F
:105F700000910023020002210348006802F0B5FBF3
:105F80000020BDE8FE8F00005487002038B50400D3
:105F9000200004F0C3F90500002D09D1200004F011
:105FA0006DFA0500002D03D1DFF8AC0C01F0E9F922
:105FB000280032BD00000810005000406487002017
:105FC0006687002070B504000D001600E4B2002CB6
:105FD00006D1320092B229006B4800F0A5FD04E022
:105FE000310089B22800FFF71BF9002302220021AB
:105FF000DFF8680C006802F02DFA70BD1C04002068
:1060000000100140F880002010B582B0040001218A
:10601000042004F0A4F84FF48070ADF800001020C4
:106020008DF8030002208DF8020000A9DFF8300C83
:1060300001F07AF8E4B2002C06D04FF48071DFF85A
:10604000200C01F029F905E04FF48071DFF8100C05
:1060500001F01FF913BD80B54FF48071DFF8000C1B
:1060600001F00AF902BD00003C87002010B586B09F
:1060700004000121A06A626B104350F0010004F09B
:106080006EF8A068DFF8DC1B884204D10121E069CA
:1060900004F065F803E00121E06904F06FF8208C5A
:1060A000ADF8040018208DF8070003208DF80600D5
:1060B00001A9606A01F038F8A08DADF80400042051
:1060C0008DF8070001A9206B01F02EF8E06802901E
:1060D000A08A002803D10020ADF80C0002E0208A3D
:1060E000ADF80C00608AADF80E00A08AADF8100083
:1060F000208BADF81400E08AADF8120002A9A06868
:1061000000F00AFF0121A06800F078FF94F83C003D
:1061100000280FD094F83C008DF8000002208DF884
:10612000010002208DF8020001208DF8030000A874
:1061300004F0A7FAA06B002818D094F83D008DF861
:10614000000002208DF8010002208DF802000120DD
:106150008DF8030000A804F094FA0121A06B03F06D
:10616000EFFF01228021A06800F081FF2021A068BC
:1061700000F090FF012240F22551A06800F04CFF92
:1061800006B010BD04ED00E0F002002088FD00081C
:106190004C050020500500205C05002068FC00082C
:1061A00070B58CB004000D001600B6B2002E2AD0D7
:1061B000B4F84C00B6B2B04225D3606C00F0B2FD2A
:1061C000A06C0090019510200290B6B203960020BA
:1061D0000490802005900020069000200790002069
:1061E00008904FF48050099000200A9000A9606C3C
:1061F00000F01DFE01220A21606C00F045FE012125
:10620000606C00F033FE0CB070BD2DE9F0438FB030
:10621000804604F075F90400A4B2002C00F09580CB
:10622000A4B240F2D370844203D3002004F07EF97C
:106230008BE0220092B2DFF8301A4FF4807004F045
:10624000F8FCA11E89B2DFF8200A03F0F1F980B250
:10625000DFF8141AA4B2611811F8011C4FF480720F
:10626000DFF8043AA4B2E31813F8023C02FB013150
:1062700088426AD10027A4B20A20B4FBF0F0FFB232
:10628000874262D2FA2001F073FC0722DFF8DC19A2
:106290000DF1260003F000F9DFF8CC090078ADF825
:1062A00022005FF000095FFA89F9B9F1030F4ADAB9
:1062B000002208A9BDF82200C0B2FFF704FD0028A3
:1062C0003BD09DF80D00DFF8A819087001208DF86B
:1062D0000C0001208DF818009DF824008DF80E00A8
:1062E000BDF822008DF80D0000208DF81700072260
:1062F0000DF1260104A803F0CFF805220DF13101BC
:106300000DF1190003F0C8F802220DF135010DF16D
:106310001E0003F0C1F802A984B06846182204F0F8
:10632000E1FC0FBC04F069F8DFF8480901F029F836
:10633000072104A801F0CAF805E0FA2001F018FCD2
:1063400019F10109AFE77F1C95E740F2D2720021F5
:10635000DFF8140903F0B0F80020040047F23050D1
:1063600001F006FC03F07EFF070001F0E1FCBFB284
:10637000DFF8041901FB07F18142EFD2DFF8FC08D6
:1063800000680600002E20D0307C01281BD17079D7
:10639000DFF8D418A4B26054B079DFF8CC18A4B2F6
:1063A00061184870F079DFF8C018A4B261188870DD
:1063B000072216F10801DFF8B008A4B22018C01CAB
:1063C00003F06AF80A343668DCE7A4B2002C1FD068
:1063D000210089B2DFF8900803F02AF90500DFF800
:1063E0008808A4B22554ADB2280ADFF87C18A4B2FC
:1063F00061184870A41C220092B2DFF86C184FF4A8
:10640000807004F0A3FB200080B204F08FF802E05B
:10641000002004F08BF803F077F99FE75403002085
:1064200010B504005FF0FF31012001F0CDFF94E8CA
:10643000070004F0C3FC962001F09AFB94E80700E3
:1064400004F0C3FCEEE700B583B0DFF8100801905C
:1064500001200090DFF8283832220021DFF82408DC
:1064600001F008FADFF82008019001200090DFF821
:106470001C3832220021DFF80C0801F0FBF9DFF8AC
:106480006405019001200090DFF8043832220021D9
:10649000DFF8F00701F0EEF9DFF850050190012078
:1064A0000090DFF8F03732220021DFF8D80701F042
:1064B000E1F9002001900320009000234FF4967230
:1064C00000210FF2C92001F0D5F90020019003202E
:1064D000009000234FF4967200210FF2155001F046
:1064E000C9F900200190022000900023C822002159
:1064F000DFF8A40701F0BEF907BD10B504002000C5
:10650000FFF7B4FD03220021012002F025FB6060AB
:106510006068002805D0002300220021606802F096
:1065200084FB6068002806D00023002200216068F8
:1065300002F056FD03E0DFF8640700F022FF10BD13
:106540006887002098FD0008F0B585B0040001A818
:10655000DFF84C17102204F0C5FBFFF77BF9002091
:10656000FFF752FD03220021012002F0F5FADFF8C7
:1065700034170860DFF82C070068002807D00023D4
:1065800000220021DFF81C07006802F04EFB002308
:1065900000220021DFF80C07006802F021FDDFF87F
:1065A0000807FFF7AAFFDFF87C05FFF7A6FFDFF873
:1065B000FC06FFF7A2FFDFF8F806FFF79EFF0120B9
:1065C00002F023FBDFF8EC160860032002F0F8FE6F
:1065D000DFF814140860DFF81004006800280FD0FA
:1065E000DFF804040168DFF8C806406802F0F2FE34
:1065F000DFF8F4030168DFF82C05406802F0EAFEDA
:10660000DFF8B40600900023002241F27071DFF839
:10661000AC0602F026F8DFF8A8160860FFF713FFB3
:1066200000235FF0FF320021DFF87806006802F0F7
:10663000D7FC002005000026F6B2042E80F09A80D8
:1066400001A8F6B250F82600C06D002857D06D1C86
:1066500001F06EFB01A9F6B251F82610C96D88420F
:106660004DD36D1E01A8F6B250F82600B0F85800C0
:1066700001A9F6B251F82610A1F85A00002001A98C
:10668000F6B251F82610A1F85800002001A9F6B280
:1066900051F82610C865F6B2002E05D0022E0DD096
:1066A00007D3032E0FD013E0DFF8180600F069FEC1
:1066B0000EE0DFF8140600F064FE09E0DFF80C06D7
:1066C00000F05FFE04E0DFF8080600F05AFEFFE786
:1066D00001A8F6B250F82600B0F85A1001A8F6B298
:1066E00050F82600006D00F0F1FE0023002200218A
:1066F00001A8F6B250F82600406802F096FA01A808
:10670000F6B250F82600006E002831D06D1C01F062
:106710000FFB070001F00CFB01A9F6B251F826109F
:10672000096E884224D36D1E002001A9F6B251F8EB
:106730002610A1F85A00002001A9F6B251F826103F
:10674000A1F85800002001A9F6B251F82610C8653A
:10675000002001A9F6B251F82610086601A8F6B289
:1067600050F82600FFF782FCDFF8680500F009FE0C
:10677000761C61E7EDB2002D02D0052001F0F8F99A
:10678000EDB2002D7FF457AF4AE700002DE9F0414C
:1067900086B004000025002604F097FBDFF83815CA
:1067A000087003F086FDDFF830050078002812D16C
:1067B0000120DFF8BC140870002302220021DFF85A
:1067C000C804006801F046FE002302220021874829
:1067D000006801F03FFE00235FF0FF320021DFF888
:1067E000C804406802F0FCFB002302220021DFF80D
:1067F0009804006801F02EFEDFF8AC04B0F85A10DF
:10680000DFF8A404006D03F017F90500002DE2D0B5
:10681000287A10F01F00C0B211281ED0132804D00F
:1068200019280ED01F2806D0CBE0DFF87C04406D7D
:10683000FEF791FEC5E0DFF87004406DFEF7C1FE83
:10684000BFE015F10A0004F045FE002804D0012144
:1068500015F10A0004F03FFDB3E000A92800FEF79F
:10686000F2FD002800F0AD809DF80000022800F045
:10687000A7800DF10600FFF789FB0600002E29D046
:10688000307C012826D1DFF82004416D00A8FFF7F5
:1068900036F9DFF81404406D03F0A2F8C0B202002C
:1068A00092B2DFF80404416DDFF8FC0300F03CF91C
:1068B000DFF8280400F065FDDFF8EC03406D03F01D
:1068C0008FF80100C9B289B2DFF8DC03406D00F037
:1068D000FDFD75E0002E07D0307C022804D1DFF8E2
:1068E000000400F04EFD6BE0DFF884030078ADF8A3
:1068F000020001F01DFA00F2E2400700002340F21E
:10690000E2420021DFF8AC03006802F069FB0028D6
:1069100004D1DFF8D00300F034FD5CE7DFF8880332
:10692000426D00A9D2480078FFF7CDF980465FFAA2
:1069300088F8B8F1000F2FD001F0FAF9874238D368
:10694000DFF86403406D03F04BF80200D2B292B25C
:10695000D548416D9DF80000FFF734FB00AA3100D7
:106960000120FFF780F9DFF8800300F00AFDCE4830
:10697000406D03F035F8C0B2010089B2CA48406DDD
:1069800000F0A4FDDFF8640300F0FBFC07210DF12B
:10699000060000F09BFD0CE000AA31000020FFF78C
:1069A00062F9D34800F0EDFC07210DF1060000F07C
:1069B0008DFD002300220021BE48006802F035F959
:1069C000FFE70021B848406802F07EF803E70000C6
:1069D000B4840020A8FD000818850020C4FE00082B
:1069E0007CFC00084C87002038870020508700205E
:1069F0002DE9F8430400002600235FF0FF32002158
:106A0000AA48406802F0ECFA99480078062802DBB0
:106A1000002001F03DF896480078002802D15FF090
:106A2000010902E0924890F8009000235FF0FF32E5
:106A300000219E48406802F0D3FA5FFA89F9B9F163
:106A4000040F03D14FF49670050009E05FFA89F94D
:106A5000B9F1030F02D14FF4967501E040F2E2451F
:106A600001F066F9060000232A0000219148006821
:106A700002F0B6FA002803D19E4800F082FCD4E769
:106A80008A48B0F85A108948006DFEF7D4FB9A483E
:106A900000F077FC8548B0F85A108448006D00F08B
:106AA00015FD01F045F9A919091A9448006802F08A
:106AB000A9FC80467E48406880451ED16C4880F81D
:106AC00000907B48B0F85A207948016D7748406DB6
:106AD00002F0E2FC7648B0F85A107548006DFEF7F7
:106AE0009BFE07003A0092B27048416D6F4800F07B
:106AF0001BF8834800F045FC0CE05D480078002856
:106B000008D15FFA89F919F10100062190FBF1F231
:106B100001FB12090023002200216648006802F0F0
:106B200084F882E71C0400202DE9F04104000D00E8
:106B30001600A0687349884223D16F4800F021FCF9
:106B4000310089B2280000F0C1FC002240F225513A
:106B50006C4800F061FAA06880894FF6FB7108402C
:106B6000A168888101F0E4F8B6B2B100323110EBCF
:106B700051002066320092B229002000FFF710FB7E
:106B800067E0A0686049884223D1604800F0F9FBC3
:106B9000310089B2280000F099FC002240F2255112
:106BA000594800F039FAA06880894FF6FB71084017
:106BB000A168888101F0BCF8B6B2B100323110EBA7
:106BC00051002066320092B229002000FFF7E8FA57
:106BD0003FE0A0682349884214D1B6B216F1640799
:106BE00001F0A6F8804601F0A3F8B6B216F1320122
:106BF00010EB51002066320092B229002000FFF70E
:106C0000CFFA26E0A0684249884221D1B6B23200CC
:106C10002900404802F05CFC00203F4908803F48C2
:106C2000068001F085F8B6B2B100323110EB5100A8
:106C30003B49086640F22661354800F031FA0028E9
:106C4000F8D1012240F22661314800F0E5F900E078
:106C5000FFE7BDE8F0810000C8FA00084487002083
:106C600000080140003801402470002027700020F7
:106C70006E870020E4FA000840771B00E4860020BD
:106C8000E00400202164000848870020EC04002074
:106C9000F8040020040500200B62000834FA000804
:106CA000F8FD00083C870020F0020020B803002017
:106CB00054030020408700208758000890FC0008FB
:106CC0005487002024FF0008B8FD00082CFF0008AE
:106CD000C8FD0008D8FD00086F870020E8FB000809
:106CE0009CF90008C0F90008A4FC0008B8FC0008E2
:106CF000CCFC0008E4F90008A8FD00083887002053
:106D000000FB000800440040004C0040E8FD000883
:106D100000500040F8800020648700206687002033
:106D20001C04002001684FF6FE7211400160002132
:106D3000016000214160002181600021C16066493D
:106D4000884206D16549096851F00F01634A116014
:106D50006CE06349884206D16049096851F0F0014E
:106D60005E4A116062E05F49884206D15B4909686A
:106D700051F47061594A116058E05B49884206D16C
:106D80005649096851F47041544A11604EE0574920
:106D9000884206D15149096851F470214F4A116067
:106DA00044E05349884206D14C49096851F47001C6
:106DB0004A4A11603AE04F49884206D1474909687A
:106DC00051F07061454A116030E04B49884206D16C
:106DD0004A49096851F00F01484A116026E04849C4
:106DE000884206D14549096851F0F001434A1160D3
:106DF0001CE04449884206D14049096851F4706159
:106E00003E4A116012E04049884206D13B49096878
:106E100051F47041394A116008E03C49884205D17B
:106E20003649096851F47021344A1160704710B432
:106E3000002203681A006FF30E128B680C6A23435A
:106E40000C6923434C6923438C692343CC69234356
:106E50004C6A23438C6A23431A430260CB68436025
:106E60000B6883604B68C36010BC7047C9B20029CF
:106E700004D0026852F00102026004E002684FF69A
:106E8000FE731A4002607047D2B2002A03D0036832
:106E90000B43036002E003688B430360704701000B
:106EA00000200022CB0003D5194B1B681A0002E01A
:106EB000184B1B681A000A4202D00123180001E097
:106EC00000231800C0B27047C10002D50B4908600A
:106ED00001E00249086070470800024004000240D7
:106EE0001C000240300002404400024058000240B2
:106EF0006C0002408000024008040240040402408A
:106F00001C04024030040240440402405804024081
:106F100000040240000002402DE9F04786B0040062
:106F20000D00002600275FF000085FF000095FF009
:106F3000000AA8890028A246208A06004CF6FF70A5
:106F40000640E88806432682A08906004EF6F31024
:106F50000640A88829890843698908430643A68111
:106F6000A08A06004FF6FF400640A8890643A68285
:106F700000A803F074F82048824502D10398070066
:106F800001E002980700A089000408D5192000FB41
:106F900007F029684900B0FBF1F0804607E01920AE
:106FA00000FB07F029688900B0FBF1F080466420FF
:106FB000B8FBF0F0000106003009642101FB1080ED
:106FC0008146A089000409D55FEAC90032306421F6
:106FD000B0FBF1F010F00700064308E05FEA09108B
:106FE00032306421B0FBF1F010F00F00064326812F
:106FF00006B0BDE8F087000000380140C9B20029A2
:1070000004D0828952F40052828104E082894DF6D4
:10701000FF731A4082817047F0B4002300240025DA
:10702000002689B240F66A17B94206000F00FFB287
:107030007F09FFB23B0089B211F01F073C00012716
:10704000A7403D00012B01D10C3604E0022B01D1F9
:10705000103600E01436D2B2002A03D037682F432E
:10706000376002E03768AF433760F0BC7047D2B298
:10707000002A03D0838A0B43838202E0838A8B43F6
:1070800083827047CA05D20D828070478088C00510
:10709000C00D704789B28A0589B2CA430280704721
:1070A00070B40200002300250024002089B240F6BD
:1070B0006A16B1420E00F6B27609F6B2340089B211
:1070C00011F01F063500012616FA05F5012C02D134
:1070D0009689354006E0022C02D1168A354001E03F
:1070E000968A354089B20E0AB6B23300012616FAE6
:1070F00003F316883340002D04D0002B02D0012664
:10710000300001E000263000C0B270BC70478268D9
:10711000521C8260426832B10268531C03601170D5
:107120004168491E41607047F0B5002700220023E6
:1071300000240025002691F803C01CF00F0C6746C0
:1071400091F803C05FEACC6C03D591F802C05CEA09
:10715000070791F800C05FEA0C6C3AD0D0F800C085
:1071600065465FF0000C6346082B31D25FF0010CDE
:107170001CFA03FC6446B1F800C014EA0C0C624629
:10718000A24223D15FEA830C64465FF00F0C1CFA25
:1071900004FC6646B54317FA04FC5CEA050591F861
:1071A00003C0BCF1280F06D15FF0010C1CFA03FCF0
:1071B000C0F814C00AE091F803C0BCF1480F05D133
:1071C0005FF0010C1CFA03FCC0F810C05B1CCBE79D
:1071D0000560B1F800C0BCF1FF0F3FDDD0F804C07E
:1071E00065465FF0000C6346082B36D25FF0010C59
:1071F00013F1080E1CFA0EFC6446B1F800C014EA44
:107200000C0C6246A24226D15FEA830C64465FF012
:107210000F0C1CFA04FC6646B54317FA04FC5CEA42
:10722000050591F803C0BCF1280F07D15FF0010CF0
:1072300013F1080E1CFA0EFCC0F814C091F803C03C
:10724000BCF1480F07D15FF0010C13F1080E1CFAD6
:107250000EFCC0F810C05B1CC6E74560F0BD020024
:107260000020936889B20B4202D00123180001E08C
:1072700000231800C0B2704702000020D36889B212
:107280000B4202D00123180001E000231800C0B215
:10729000704789B20161704789B241617047F0B4AB
:1072A0000022002300250024002803D51E4E366846
:1072B000350002E01D4E36683500C0F30346340049
:1072C00086B2320010F44016B6F5401F08D135F0F2
:1072D0007065164E366836F07066144F3E6010E0EA
:1072E000C60206D50326A64033009D4355F07065BF
:1072F00007E0460DF6B2360112FA06F6B54355F030
:107300007065C9B2002905D0460DF6B2360112FAF1
:1073100006F63543002802D5034E356001E0034EE2
:107320003560F0BC704700001C00014004000140C3
:107330000020DFF8E814087070470120DFF8DC1443
:107340000870704738B504000D00EDB22A0092B203
:107350002100DFF8CC04FEF723FF31BD80B5FF220A
:107360000021DFF8BC04006D02F0A6F80020DFF871
:10737000B014A1F85A0001BDDFF8A404B0F85A0017
:1073800070470EB430B50400DFF890040078002890
:1073900000F09680FF220021DFF8880402F08CF8CC
:1073A00003A8DFF884140860DFF87C040368220077
:1073B000FF21DFF8700404F087FADFF8701408800A
:1073C0000020DFF86C140870DFF8600400880028E3
:1073D00076D0DFF858040088FF2871DCDFF84C0411
:1073E0000088142190FBF1F201FB1200002809D162
:1073F000DFF838040088142190FBF1F0DFF8341432
:10740000087009E0DFF824040088142190FBF1F0F3
:10741000401CDFF82014087004F0DAFA0025DFF8C9
:1074200014040078EDB2854248D2EDB2DFF80404CE
:107430000078401E854217D1DFF8F0030088142140
:1074400090FBF1F201FB1200002801D1142007E0AB
:10745000DFF8D8030088142190FBF1F201FB120041
:10746000DFF8D413087003E01420DFF8CC130870A1
:10747000DFF8C4030078DFF8C41308701422DFF8C3
:10748000A403DFF8AC1309780918DFF8B40302F09D
:1074900003F8DFF89C030078DFF89C1309780818DC
:1074A000DFF88C13087000230022DFF89013DFF858
:1074B0009403006801F0B9FB6D1CB0E704F0A3FA77
:1074C000DFF88403008830BC5DF810FB2DE9F04143
:1074D00004000D005FF00008122614220021DFF8DE
:1074E0006C0301F0E9FF04F073FA00273800C0B222
:1074F00080B2ADB2A8425AD2404610F10108FFB2A4
:10750000395D102291FBF2F10A2906DAFFB2395DEA
:10751000102291FBF2F1303105E0FFB2395D10220B
:1075200091FBF2F15731C94AC0B28154404610F183
:107530000108FFB2395D102291FBF2F303FB121335
:107540000A2B09DAFFB2395D102291FBF2F303FB3B
:10755000121313F1300108E0FFB2395D102291FBE4
:10756000F2F303FB121313F15701B84AC0B281546E
:107570002020B6495FFA88F808F8010018F10108E0
:107580005FFA88F8F6B2B04504D2FFB2ADB2681E19
:1075900087420AD100208046AC4958A0FFF7F1FE8F
:1075A00014220021A94801F087FF7F1C9EE79AA0C2
:1075B000FFF7E7FE04F027FABDE8F08110B586B0CA
:1075C000040000235FF0FF3200A99E48006801F02C
:1075D00007FD0128F5D19DF8002092B20DF10101BF
:1075E0008F48FEF7DDFD00234FF47A7200219848A2
:1075F000006801F0F5FC0028E3D18948FEF736FD6C
:1076000000208749A1F8580000208549A1F85A00B8
:10761000D7E710B5040000235FF0FF320021804857
:10762000406801F0DDFC0128F5D104F05FFAFFF7B6
:1076300095FEF0E700B583B07948FEF717FD00220C
:107640001521C82001F088FA7E4908600322002134
:10765000012001F081FA7E4908607D480068002819
:1076600006D00023002200217948006801F0DDFAED
:1076700000217748006801F027FA6948FEF73DFFCE
:1076800000200190052000900023C8227149724813
:1076900000F0F0F800200190022000900023C822A2
:1076A0006E496F4800F0E6F86E48FFF76AFE07BDC6
:1076B00080B5002000902020FFF7F1FB002813D0B8
:1076C0002020FFF701FC00A96148006801F013FCCD
:1076D0000098002810D05FF0805063490860BFF325
:1076E0004F8FBFF36F8F07E08020FFF7D8FB002894
:1076F00002D08020FFF7E8FB01BD000025730000E9
:1077000030B585B001A85949102203F0EBFA0020EA
:10771000009040F225515648FFF7C2FC002879D06E
:107720005348FFF7B3FC05003D48B0F85800FF2868
:1077300003DB00203A49A1F85800EDB2082D22D110
:107740000B223748016D01A801F0CAFF00280DD0B7
:107750003348006D3249B1F858100D543048B0F834
:107760005800401C2E49A1F8580053E02C48B0F8AE
:10777000580000284ED02A48B0F85800401E28492A
:10778000A1F8580046E02648006D2549B1F8581088
:107790000D542348B0F85800401C2149A1F8580066
:1077A000EDB20D2D02D0EDB20A2D33D10B221C48C3
:1077B000016D01A801F094FF002811D01848006D58
:1077C000007B1749096D497B4FF4807202FB010071
:1077D0000F3004001248B0F85800A4B2A04219D3E8
:1077E0000F48B0F858000E49A1F85A0000200C4983
:1077F000A1F8580000A90A48406801F07CFB0098F5
:10780000002807D05FF0805017490860BFF34F8F02
:10781000BFF36F8F05B030BD0D0A00006305002077
:107820008C020020F8780020CC86002060870020A1
:107830006B8700206A8700206C870020C4850020A9
:10784000C5850020C486002062870020F4850020C2
:10785000C886002088FE0008BD75000828FD0008C5
:107860001376000894FE000804ED00E038FD0008DF
:10787000004800402DE9F04F85B004000D001600CF
:107880001F00DDF83880DDF83C90B6B2B00004F09F
:10789000ADFC8346BBF1000F0DD05C2004F0A6FCCC
:1078A0008246BAF1000F02D0CAF830B005E058465F
:1078B00004F022FD01E000208246BAF1000F14D04E
:1078C00000200390CDF808A0CDF80490CDF80080FA
:1078D0003B00B6B232002900200000F00DF85046FF
:1078E00000F076F80120049002E05FF0FF30049091
:1078F000049805B0BDE8F08F2DE9F94F83B00C0076
:1079000015000E9E0F9FDDF84080A8000190A52075
:107910000090D8F830B0009A0199584604F09CFDC8
:10792000D8F8300010EB8500001F81465FEAD909C6
:107930005FEAC90919F00700002805D0DFF8DC1656
:1079400040F22B3004F040FE00208246BAF1100FC6
:107950000CD21AF804001AEB080181F834001AF866
:107960000400002802D01AF1010AEFE7002088F88D
:107970004300052E01D304200600C8F82C60C8F887
:107980004C600020C8F8500018F1040004F03BFEE1
:1079900018F1180004F037FEC8F81080D6F1050081
:1079A000C8F81800C8F824800020C8F85400002047
:1079B00088F85800049A0399484603F0A3FFC8F8D2
:1079C0000000002F01D0C7F8008005B0BDE8F08F9F
:1079D00010B5040003F0FCFFDFF868050068401CE8
:1079E000DFF860150860DFF86005006800280AD13C
:1079F000DFF854050460DFF84C050068012811D158
:107A000000F08CFB0EE0DFF844050068002809D187
:107A1000E06ADFF834150968C96A884202D3DFF8E2
:107A200028050460DFF828050068401CDFF82015F1
:107A30000860DFF81C0500686064DFF8180500685E
:107A40000121E26A91400843DFF808150860211D12
:107A5000DFF80405E26A142303FB020004F0D6FDFC
:107A600003F0D1FFDFF8E404006800280FD0DFF84E
:107A7000D8040068C06AE16A884208D25FF080508A
:107A8000DFF860160860BFF34F8FBFF36F8F10BD34
:107A900038B5040003F09CFF002C03D1DFF8A804E4
:107AA000056800E02500281D04F0D9FD002812D14A
:107AB000DFF8A404E96A142202FB01000068002830
:107AC00009D1DFF8900400680121EA6A91408843F7
:107AD000DFF880140860A86A002803D015F11800A8
:107AE00004F0BDFDDFF868040068401CDFF8601496
:107AF0000860DFF85404006885420CD1291DDFF8C6
:107B0000200504F083FDDFF81C050068401CDFF849
:107B1000141508600BE0DFF82C040068401EDFF845
:107B200024140860280000F059FB00F060FB03F00B
:107B30006AFFDFF818040068002818D0DFF808048E
:107B40000068854213D1DFF8E0040068002805D002
:107B5000DFF8C81440F2654004F036FD5FF0805055
:107B6000DFF880150860BFF34F8FBFF36F8F31BD13
:107B700038B504000025002C13D0DFF8AC040068F1
:107B8000002805D0DFF8941440F2CF4004F01CFD2B
:107B900000F04AF80021200000F0DEFC00F04CF874
:107BA0000500002D08D15FF08050DFF8381508601F
:107BB000BFF34F8FBFF36F8F31BD1CB5DFF8FC07EC
:107BC00001900020009000234622DFF8F4170FF206
:107BD0002150FFF74FFE0400012C02D100F020FDE0
:107BE0000400012C16D1102080F31188BFF34F8FB1
:107BF000BFF36F8F5FF0FF30DFF8C8170860012018
:107C0000DFF8481308600020DFF82014086003F054
:107C10009BFE08E014F1010F05D1DFF8001440F2DB
:107C2000847004F0D1FC13BDDFF8FC030068401C35
:107C3000DFF8F4130860704770B500240025DFF802
:107C4000E8030068002805D1DFF8D0134FF4FD6089
:107C500004F0BAFC03F0BCFEDFF8CC030068401E61
:107C6000DFF8C4130860DFF8C003006800285BD1A8
:107C7000DFF8D0020068002856D0DFF8D00700688F
:107C8000002829D0DFF8C407C068C068040014F1D8
:107C9000180004F0E4FC201D04F0E1FCDFF8B4025D
:107CA00000680121E26A91400843DFF8A8120860E9
:107CB000211DDFF8A402E26A142303FB020004F092
:107CC000A5FCE06AA0490968C96A8842D5D30120A9
:107CD000DFF878180860D0E7002C01D000F087FAB0
:107CE000DFF86C070668002E0ED000F026F800289A
:107CF00003D00120DFF854180860761E002EF4D15E
:107D00000020DFF84C170860DFF840080068002802
:107D10000AD0012005005FF08050DFF8C81308602A
:107D2000BFF34F8FBFF36F8F03F06DFE280070BD60
:107D3000DFF8F8120968080070472DE9F0410026C5
:107D4000B9480068002840F08180DFF8E002006850
:107D5000471CDFF8D8020760002F21D1DFF8880325
:107D600000680068002804D0AC4940F6D91004F03F
:107D70002BFCDFF8740300688046DFF870030068AE
:107D8000DFF864130860DFF86403C0F80080DFF8F0
:107D9000C0070068401CDFF8B817086000F027FA39
:107DA000DFF82006006887423CD3DFF83C03006818
:107DB0000068002805D15FF0FF30DFF80816086082
:107DC00030E0DFF824030068C068C0680400606821
:107DD0000500AF4203D2DFF8EC05056022E0201D6C
:107DE00004F03DFCA06A002803D014F1180004F050
:107DF00036FC584800680121E26A91400843554921
:107E00000860211D5448E26A142303FB020004F0B9
:107E1000FDFBE06A4C490968C96A8842C5D3012064
:107E20000600C2E74C4848490968C96A142202FBA7
:107E300001000068022801D301200600DFF81006C7
:107E4000006800280BD104F0BDFB08E0DFF8000655
:107E50000068401CDFF8F815086004F0B3FBDFF899
:107E6000EC060068002801D0012006003000BDE8C3
:107E7000F08138B56C480068002804D00120DFF894
:107E8000CC16086045E00020DFF8C01608602E48D8
:107E90000068006B05005FF0A53004002868A04270
:107EA00008D16868A04205D1A868A04202D1E8685C
:107EB000A04207D02448006810F13401224800682D
:107EC00004F078FB23480068B0FA80F0D0F11F007E
:107ED00004002148142101FB04000068002804D19B
:107EE0004E4940F6F62004F06FFB1B49142202FBBA
:107EF00004110800416849684160416810F10802B6
:107F0000914202D14168496841604068C0680E49A9
:107F1000086031BD38B504000D00002C04D13F4984
:107F200040F6063004F050FBDFF8B006006810F1B0
:107F30001801200004F076FB0121280000F00CFB62
:107F400031BD0000F8860020E8860020048700206C
:107F50001487002000870020EC83002070B5040007
:107F60000D001600002C04D12C4940F6313004F0ED
:107F70002BFBDFF86806006810F11801200004F000
:107F800045FB002E02D05FF0FF30050031002800D5
:107F900000F0E2FA70BD70B50400E068C06805004A
:107FA000002D04D11D4940F6613004F00DFB15F1A0
:107FB000180004F054FB1C480068002816D1281D46
:107FC00004F04DFBDFF8180600680121EA6A9140D1
:107FD0000843DFF80C160860291DDFF80806EA6A76
:107FE000142303FB020004F011FB05E015F1180156
:107FF000DFF8580404F00AFBDFF8E0050068C06A07
:10800000E96A884206D2012006000120DFF8441503
:10801000086001E000200600300070BD10F9000883
:1080200044860020F486002020870020FC86002063
:1080300010B50400002C05D1DFF8B01540F6C130B2
:1080400004F0C2FADFF8080500682060DFF8A00538
:108050000068606010BDF8B504000D00002C05D16B
:10806000DFF8881540F6CB3004F0AEFA002D05D1CC
:10807000DFF8781540F6CC3004F0A6FA03F0A8FC3F
:10808000DFF86C050768286810F1010F02D10020A5
:1080900006001DE0DFF8B80400682168884205D0BA
:1080A0006068874202D30120060011E06068381A38
:1080B000296888420AD22868C01B616808182860AD
:1080C0002000FFF7B5FF0020060001E001200600B8
:1080D00003F099FC3000F2BD0120DFF8781408604D
:1080E0007047000004ED00E0EC860020F0860020E0
:1080F00010B5040000F03FF8DFF8E804006802283B
:1081000008D35FF08050DFF8EC140860BFF34F8FA6
:10811000BFF36F8F04F04DFAECE7000010B50020BC
:108120000400052C08D2DFF8BC04142101FB040074
:1081300004F05AFA641CF4E7DFF8BC0404F054FAC3
:10814000DFF8B80404F050FADFF8000304F04CFA4A
:10815000DFF8AC0404F048FADFF8A80404F044FAAD
:10816000DFF89404DFF8A0140860DFF89004DFF86B
:108170009C14086010BD38B5DFF89404006800282E
:108180002BD0FFF751FDDFF878040068002801D1FB
:10819000012400E00024FFF74FFD002CECD103F098
:1081A00017FCDFF85C04C068C0680500281D04F0F7
:1081B00056FADFF860040068401EDFF858140860C3
:1081C000DFF84C040068401EDFF84414086003F038
:1081D0001AFC280000F002F8CEE731BD10B504000B
:1081E000206B04F089F8200004F086F810BDDFF859
:1081F000181409680968002904D15FF0FF31714A39
:10820000116008E0DFF800140968C968C96808004F
:1082100041686C4A11607047DFF8FC130968002957
:1082200002D10121080009E0DFF8BC130968002928
:1082300002D10221080001E000210800704738B592
:1082400004002500002C4FD0E86ADFF8901309687D
:10825000C96A884248D2A869002806D4DFF87C039E
:108260000068C06AD0F10500A8616869DFF874137E
:10827000EA6A142303FB0211884230D1281D04F05E
:10828000EEF9002812D1DFF85C03E96A142202FB40
:1082900001000068002809D1DFF8440300680121CB
:1082A000EA6A91408843DFF838130860DFF82C034E
:1082B0000068C06AE862DFF8280300680121EA6A02
:1082C00091400843DFF818130860291DDFF81403F4
:1082D000EA6A142303FB020004F098F904E0DFF8D3
:1082E000FC020068C06AE86231BD70B50400250078
:1082F0000026002C50D0DFF8E4020068854205D04B
:10830000DFF8E81240F6C76004F05EF9286D002837
:1083100005D1DFF8D81240F6C96004F055F9286D90
:10832000401E2865E86AE96C884235D0286D00282F
:1083300032D1281D04F093F9002812D1DFF8A402ED
:10834000E96A142202FB01000068002809D1DFF865
:10835000900200680121EA6A91408843DFF88012A8
:108360000860E86CE862E86AD0F10500A861DFF80F
:10837000700200680121EA6A91400843DFF8601248
:108380000860291DDFF85C02EA6A142303FB02007F
:1083900004F03CF901200600300070BDDFF83C021B
:1083A0000068002805D0DFF834020068016D491C20
:1083B0000165DFF828020068704700001C87002074
:1083C0000CFF00081887002070B504000D0003F0B2
:1083D000FFFADFF808020068406D002814D1012080
:1083E000DFF8F811096881F85800002D0CD0012140
:1083F000280000F0B1F85FF08050DFF8F811086055
:10840000BFF34F8FBFF36F8F03F0FDFA03F0E0FA75
:10841000DFF8C8010068406D0600002E0CD0002C6B
:1084200005D00020DFF8B4110968486504E0701E2B
:10843000DFF8A811096848650020DFF8A011096875
:1084400081F8580003F0DFFA300070BD308600205C
:10845000088700202DE9F04704000D0016001F00DA
:108460005FF00109002C05D1DFF8801141F2FD0019
:1084700004F0AAF8A04603F0ABFA002F02D0D8F817
:108480005400386098F858008246022088F8580056
:10849000F6B2002E20D0022E0AD003D3042E10D024
:1084A0000CD319E0D8F854002843C8F8540013E05E
:1084B000D8F85400401CC8F854000DE0C8F85450D7
:1084C0000AE05FFA8AFABAF1020F02D0C8F85450F3
:1084D00001E000208146FFE75FFA8AFABAF1010F56
:1084E0002ED118F1040004F0BAF83D4800680121CB
:1084F000D8F82C20914008433949086018F104014C
:108500003848D8F82C20142303FB020004F07EF82E
:10851000D8F82800002804D0344941F2351004F07E
:1085200053F82E480068C06AD8F82C10884207D249
:108530005FF080502F490860BFF34F8FBFF36F8FFC
:1085400003F061FA4846BDE8F08700000C87002080
:10855000108700200C870020F8B504000D00244887
:1085600007681E480068001D04F079F800280BD148
:108570001A4800681A4909680122C06A12FA00F014
:1085800031EA00001649086014F1010F08D1002DEE
:1085900006D012480068011D1A4804F037F81BE0A5
:1085A000E01906000D4800684660BE4207D20B483D
:1085B0000068011D1548006804F034F80CE0074815
:1085C0000068011D1048006804F02CF8134800688A
:1085D000864201D211480660F1BD0000E886002005
:1085E00000870020EC8300202087002010F900087D
:1085F000FC86002004ED00E0088600201C86002098
:108600004486002058860020EC860020F08600205A
:10861000F4860020F88600200487002018870020B8
:108620001CB5002400F014FADFF87004006800287C
:108630000DD0DFF86C040190042000900023462246
:10864000DFF860140FF27D10FFF714F90400002C1E
:1086500005D1DFF8541440F2331003F0B5FF2000C9
:1086600016BD2DE9F04383B004000D0016001F0075
:10867000DDF828802C2003F0B9FD8146B9F1000F08
:1086800009D0CDF80490CDF800803B0032002900DD
:10869000200000F003F84846BDE8FE832DE9F843CA
:1086A00004000D0016001F00DDF82080DDF8249086
:1086B000002D05D1DFF8F0134FF4C67003F084FFEE
:1086C000B9F1000F0FD000F0C3F9C9F80040C9F8A4
:1086D0001850C9F81C60C9F82070C9F8248019F135
:1086E000040003F090FFBDE8F1832DE9FE43040090
:1086F0000D0016001F00DDF828805FF00009002C37
:1087000005D1DFF8A4134FF4D37003F05DFFDFF859
:108710008C030068002825D0009501960294062D50
:1087200017DAFFF779FD022809D10023424600A994
:10873000DFF86803006800F078FA814612E0002351
:10874000002200A9DFF85403006800F06EFA8146A9
:1087500008E000233A0000A9DFF84003006800F0B9
:108760004AFB81464846BDE8FE83F8B504000D008B
:10877000DFF838030068C068C768381D03F06FFF72
:10878000F869012819D123002A00B86901193800B5
:1087900000F088F8002810D000200090002322006C
:1087A00000213800FFF7A1FF0600002E05D1DFF8F9
:1087B000F8124FF4027003F007FF3800796A884717
:1087C000F1BD000038B5040000A800F040F8050035
:1087D0000099280000F003F800F08CF8F4E770B579
:1087E00082B004000E00FFF71FFA00A800F046F860
:1087F00005000098002827D1002E08D1A54206D3F5
:10880000FFF71AFA29002000FFF7AFFF1EE0002E45
:1088100007D0A74800680068002801D1012600E0C1
:1088200000263200611B9D48006800F0A3FDFFF7A1
:1088300003FA00280AD15FF080509E490860BFF318
:108840004F8FBFF36F8F01E0FFF7F6F973BD0100A3
:10885000964A12681268002A01D1012200E0002223
:10886000D2B20A600A68002A05D1904A1268D2681A
:108870001268100001E000221000704738B50400B3
:10888000FFF756FA05008C480068854204D200F0D4
:108890009AF80120206001E00020206086480560F1
:1088A000280032BD2DE9F04104000D0016001F0024
:1088B0005FF0000865602461AE420CD3F01BA16933
:1088C000884202D30120804611E0211D78480068CB
:1088D00003F0A8FE0BE0BE4204D2BD4202D3012049
:1088E000804604E0211D7148006803F09BFE40466D
:1088F000BDE8F08170B586B00023002201A9674869
:10890000006800F06DFB00285BD001980028F3D4CC
:10891000039804006069002802D0201D03F09FFE28
:1089200004A8FFF7ABFF0600019800280ED002282C
:108930000CD00BD304282DD02BD3062806D03BD344
:10894000082826D002D3092824D039E0029B32001F
:108950000298A16909182000FFF7A4FF002817D08A
:108960002000616A8847E069012811D10020009049
:1089700000230298A1690A1800212000FFF7B5FE24
:108980000500002D04D1484940F2213003F01CFEBF
:10899000B2E7B1E70298A061A069002804D142497A
:1089A0004FF44E7003F010FE33003200A0698119BD
:1089B0002000FFF777FF9FE7200003F09DFC9BE777
:1089C0009AE706B070BD2DE9F04182B037480068E3
:1089D0000068002831D035480068C068006804008D
:1089E00032480068C068C0680700381D03F037FED1
:1089F0003800796A8847F8690128E7D1B869001911
:108A00000500AC4207D27D603F61391D27480068F0
:108A100003F008FEDAE70020009000232200002186
:108A20003800FFF762FE8046B8F1000F04D11E49FE
:108A300040F2923003F0C8FDC8E71C480068060009
:108A40001B4800681949086019480660BDE8F381B1
:108A500080B502F0BDFF1148006800281BD11748FF
:108A600003F0C2FD164803F0BFFD14480F4908602B
:108A700013480F49086000220C210A2000F06CF80E
:108A80000649086005480068002804D00D490348DD
:108A9000006800F058FC02F0B6FF01BD2C870020F2
:108AA0003087002014FF0008A4F800082487002065
:108AB0002887002004ED00E0348700206C86002029
:108AC000808600201CFF000870B504000D00260001
:108AD000002E05D1DFF8981840F21B1003F074FD4A
:108AE00002F076FF3068F16B326C02FB01007060BF
:108AF0000020B0633068B0603068F16B491E326CA2
:108B000002FB0100F0605FF0FF3086F844005FF088
:108B1000FF3086F84500002D12D13069002817D0AB
:108B200016F11000FFF737FA002811D05FF08050DF
:108B3000DFF858190860BFF34F8FBFF36F8F07E05E
:108B400016F1100003F050FD16F1240003F04CFD67
:108B500002F059FF012070BD2DE9F84304000D001B
:108B60001600002C05D1DFF808184FF4C47003F08C
:108B70002BFD002D02D10020804602E005FB04F011
:108B8000804618F1540003F031FB0700002F0AD093
:108B900017F15400814600973300DBB24A462900A2
:108BA000200000F003F83800BDE8F2832DE9F04121
:108BB00004000D0016001F00DDF81880002D02D102
:108BC000C8F8008001E0C8F80060C8F83C40C8F868
:108BD000405001214046FFF777FF88F85070002091
:108BE000C8F84800BDE8F08110B50400002C0BD097
:108BF00000206060002020600020E0600023002250
:108C00000021200000F011F810BDF8B50400012685
:108C100000272200D2B239003000FFF79DFF050087
:108C20002800FFF7E1FF2800F2BD2DE9F74304001B
:108C30000D001E005FF00008A146B9F1000F05D13C
:108C4000DFF82C1740F2D92003F0BEFC002D03D131
:108C5000D9F84000002801D1012000E00020C0B276
:108C6000002805D1DFF8081740F2DA2003F0ACFC49
:108C7000022E03D1D9F83C00012801D1012000E0E7
:108C80000020C0B2002805D1DFF8E41640F2DB2056
:108C900003F09AFCFFF7C0FA002802D102980028DE
:108CA00001D1012000E00020C0B2002805D1DFF88A
:108CB000C01640F2DE2003F087FC02F089FED9F8EE
:108CC0003800D9F83C10884201D3022E3CD1320042
:108CD0002900484600F06CFA0700D9F8480000283F
:108CE0000FD03100484600F09AFB002828D05FF0F2
:108CF0008050DFF898170860BFF34F8FBFF36F8F76
:108D00001EE0D9F8240000280FD019F12400FFF745
:108D100042F9002814D05FF08050DFF87017086027
:108D2000BFF34F8FBFF36F8F0AE0002F08D05FF0C3
:108D30008050DFF858170860BFF34F8FBFF36F8F75
:108D400002F061FE012054E00298002803D102F0F5
:108D50005AFE00204DE0B8F1000F04D100A8FFF743
:108D600067F90120804602F04EFEFEF75DFF02F03B
:108D70002FFE99F9440010F1010F02D1002089F86B
:108D8000440099F9450010F1010F02D1002089F843
:108D9000450002F038FE02A900A8FFF75CF90028A0
:108DA00021D1484600F0BEFA002816D0029919F1E8
:108DB0001000FFF7AFF8484600F05FFAFEF73CFFFF
:108DC00000287FF47AAF5FF08050DFF8C0160860AB
:108DD000BFF34F8FBFF36F8F6FE7484600F04DFA38
:108DE000FEF72AFF69E7484600F047FAFEF724FF3E
:108DF0000020BDE8FE832DE9F84F04000D001600A9
:108E00001F00A246BAF1000F05D1DFF8641540F249
:108E10009F3003F0D9FB002D03D1DAF84000002881
:108E200001D1012000E00020C0B2002805D1DFF808
:108E300040154FF4687003F0C7FB022F03D1DAF836
:108E40003C00012801D1012000E00020C0B2002830
:108E500005D1DFF81C1540F2A13003F0B5FB02F09C
:108E60000BFEEFF311808146102080F31188BFF3D1
:108E70004F8FBFF36F8FDAF83800DAF83C10884272
:108E800001D3022F30D19AF945B03A00290050465B
:108E900000F08EF94FFA8BFB1BF1010F1DD1DAF8B0
:108EA000480000280AD03900504600F0B8FA0028DF
:108EB00017D0002E15D00120306012E0DAF824001F
:108EC00000280ED01AF12400FFF765F8002808D01A
:108ED000002E06D00120306003E01BF101008AF86B
:108EE00045000120804601E00020804689F311887A
:108EF0004046BDE8F28F2DE9F04704000D00A04682
:108F0000B8F1000F05D1DFF8681440F23C4003F0DF
:108F10005BFBD8F84000002805D0DFF854144FF46C
:108F2000886003F051FBD8F80000002803D1D8F87E
:108F30000400002801D1012000E00020C0B2002878
:108F400005D1DFF82C1440F2454003F03DFB02F060
:108F500093FDEFF311800700102080F31188BFF319
:108F60004F8FBFF36F8FD8F83890D8F83C00814509
:108F70002FD298F945A019F10100C8F838004FFA2E
:108F80008AFA1AF1010F1DD1D8F8480000280AD03A
:108F90000021404600F043FA002817D0002D15D0DC
:108FA0000120286012E0D8F8240000280ED018F123
:108FB0002400FEF7F0FF002808D0002D06D0012085
:108FC000286003E01AF1010088F84500012006003E
:108FD00001E00020060087F311883000BDE8F0872B
:108FE0002DE9F44783B004000D001E000027A146C0
:108FF000B9F1000F05D1DFF8781340F2DC4003F03F
:10900000E3FA002D03D1D9F84000002801D1012056
:1090100000E00020C0B2002805D1DFF8541340F270
:10902000DD4003F0D1FAFFF7F7F8002802D10398EA
:10903000002801D1012000E00020C0B2002805D1A5
:10904000DFF82C134FF49C6003F0BEFA02F0C0FC72
:10905000D9F838A0BAF1000F41D0D9F80C008046F9
:109060002900484600F0F1F8002E1FD1BAF10100A6
:10907000C9F83800D9F80000002803D1FFF78EF9AD
:10908000C9F80400D9F81000002824D019F1100004
:10909000FEF781FF00281ED05FF08050DFF8EC1350
:1090A0000860BFF34F8FBFF36F8F14E0C9F80C80D7
:1090B000D9F8240000280ED019F12400FEF76BFF28
:1090C000002808D05FF08050DFF8C0130860BFF3BD
:1090D0004F8FBFF36F8F02F096FC012065E003987D
:1090E000002803D102F08FFC00205EE0002F04D1A5
:1090F00000A8FEF79DFF0120070002F084FCFEF7A8
:1091000093FD02F065FC99F9440010F1010F02D1C2
:10911000002089F8440099F9450010F1010F02D1AF
:10912000002089F8450002F06EFC03A900A8FEF7B4
:1091300092FF00282DD1484600F0E4F8002822D004
:10914000D9F80000002807D102F042FCD9F8040049
:10915000FFF775F802F057FC039919F12400FEF7A8
:10916000D9FE484600F089F8FEF766FD00287FF436
:109170006DAF5FF08050DFF814130860BFF34F8FBE
:10918000BFF36F8F62E7484600F077F8FEF754FDB3
:109190005CE7484600F071F8FEF74EFD484600F0E7
:1091A000B1F800283FF452AF002004B0BDE8F087CA
:1091B0002DE9F04704000D0016000027A06B804643
:1091C000206C002809D12068002838D16068FFF79A
:1091D0008CF807000020606031E0002E13D1D4F835
:1091E0004090D4F808A04A462900504601F06AFD94
:1091F000A068216C0818A060A068616888421ED32E
:109200002068A0601BE0D4F84090D4F80CA04A4637
:109210002900504601F056FDE068216C401AE060DC
:10922000E0682168884203D26068216C401AE060DF
:10923000022E04D1B8F1000F01D0B8F1010818F1E5
:109240000100A0633800BDE8F087F8B504000D0008
:10925000206C002810D0E068216C0818E060E068FD
:109260006168884201D32068E060266CE7683200BC
:109270003900280001F026FDF1BD70B5040002F0B0
:10928000A7FB94F945506DB2012D1ADBA06C0028A4
:1092900008D00021200000F0C2F800280FD0FEF70F
:1092A0001BFF0CE0606A002808D014F12400FEF7D0
:1092B00072FE002803D0FEF70FFF00E001E06D1EF4
:1092C000E1E75FF0FF3084F8450002F09CFB02F01C
:1092D0007FFB94F9446076B2012E0CDB20690028F4
:1092E00009D014F11000FEF756FE002801D0FEF759
:1092F000F3FE761EEFE75FF0FF3084F8440002F0E3
:1093000082FB70BD38B5040002F062FBA06B002840
:1093100002D10120050001E00020050002F073FBEE
:10932000280032BD38B5040002F052FBA06BE16B9F
:10933000884202D10120050001E00020050002F072
:1093400062FB280032BD00231A00052A0ED2504BC2
:1093500053F83230002B07D14D4B43F832104C4BB1
:1093600013EBC203586001E0521CEEE770470000A7
:10937000DCF80008F8B504000D001600270002F024
:1093800027FB97F9440010F1010F02D1002087F864
:10939000440097F9450010F1010F02D1002087F831
:1093A000450002F030FBB86B002805D132002900DF
:1093B00017F12400FEF7D2FD3800FFF75EFFF1BD84
:1093C00038B50400002204212000FFF7C5FB05008A
:1093D000280032BD70B504000D0002F0F9FAA06C4F
:1093E000002802D00020060008E0A06B002802D070
:1093F0000020060002E0A5640120060002F003FB45
:10940000300070BD38B504000D000020009000232E
:109410002A0000A92000FFF7E3FD009832BDF1B556
:109420000C000098856C0026002D04D1194940F6E7
:10943000CE1003F0C9F8A86BE96B884204D3154934
:1094400040F6CF1003F0C0F8A86BE96B88421AD23F
:1094500095F94570220000A92800FFF7A9FE060033
:109460007FB217F1010F0BD1686A00280BD015F1FC
:109470002400FEF790FD002805D00120060002E040
:10948000781C85F845003000F2BD000004ED00E0D6
:109490007C850020DCF8000830B4030018000C00C4
:1094A00015006A1EADB2002D04D025780570641C2D
:1094B000401CF5E730BC704710B403001400621E76
:1094C000A4B2002C02D019705B1CF7E710BC7047E7
:1094D00030B40B00040015006A1E002D04D01D7866
:1094E00025705B1C641CF6E730BC704710B40300A9
:1094F0001400621E002C02D019705B1CF8E710BC2F
:109500007047109010B5040006223E49200000F07C
:10951000E7F8002801D0012012E006223A49200095
:1095200000F0DEF8002801D0022009E006223749C9
:10953000200000F0D5F8002801D0032000E0002032
:1095400010BD30B583B004000020C0B206280DDA8B
:10955000C0B2211A49792B4AC0B28154C0B2211A33
:10956000497900AAC0B28154401CEEE70621254883
:1095700000F05EF8050028008DF80600ADB2280A5C
:109580008DF80700224803F07FF8002804D1082254
:1095900000A91F4803F095F837BD30B583B004002B
:1095A00008221B4900A8FFF793FF062100A800F03E
:1095B0003FF80500ADB29DF806009DF807104FF486
:1095C000807202FB0100854206D1062200A920001C
:1095D000FFF77EFF012005E006220A492000FFF781
:1095E00077FF00203EBD00B583B000A8FFF7D5FF90
:1095F000002805D0062200A90248FFF769FFFFE70F
:1096000007BD000038050020280500203005002097
:10961000004C0008BFF34F8F2348006810F4E0604F
:109620002249084320490860BFF34F8F00BFFDE780
:1096300030B402004FF6FF700B00591E9BB2002B96
:109640000CD080B21A4B0400A4B215786C40E4B27E
:1096500033F8143093EA1020521CEDE780F47F4079
:1096600090F0FF0080B230BC704730B40200FF20A1
:10967000FF230D00691EADB2002D0ED0C0B21578CB
:1096800045402C00521C0B4DA4B2655D5D40280086
:10969000094DA4B2655D2B00EBE7DBB2C0B250EA26
:1096A000032080B230BC70470CED00E00400FA05E6
:1096B000D8F20008000000200001002010B40200D1
:1096C000002000231C00E4B2A4B289B28C4204D270
:1096D000DBB29C5C20185B1CF4E7C0B210BC704786
:1096E00030B403000020C0B2D2B2904209D2C0B25E
:1096F000C45CC0B2455CAC4201D0002002E0401C1A
:10970000F1E7012030BC704780B5012080F3138859
:10971000FFF780FF01BD00000100002000231A00B8
:10972000082A12DAC0B2C9B291EA0003DB0706D5F3
:1097300090F01800C0B2400850F0800001E0C0B2C4
:109740004008C9B24908521CEAE7C0B2704770B578
:1097500004000D0000262800451E80B2002807D016
:1097600020787040C0B2FFF7D7FF0600641CF2E714
:109770003000C0B270BD10B40622D2B2C9B28B1E86
:109780009A420ADAD2B2135CD2B2141814F8014C1D
:109790006340D2B21354521CEFE710BC704770B54F
:1097A0008EB004000D000026682000A9F6B27054A7
:1097B000761C0120C0B2EDB2691E884221DAC0B227
:1097C000015D682907D0C0B2015D162903D0C0B27F
:1097D000015D7D290DD17D2100AAF6B2B154761C20
:1097E000C0B2015D91F0200100AAF6B2B154761C1E
:1097F00005E0C0B2015D00AAF6B2B154761C401C6F
:10980000D8E7162000A9F6B27054761CF6B23200E2
:1098100092B200A92000FFF73FFE3000C0B20EB0A8
:1098200070BD2DE9F84304000D00681EC0B20A287F
:1098300008D3C0B2015D162902D1401C804601E068
:10984000401EF3E75FFA88F8B8F10A0F01D2002052
:1098500066E05FF000095FFA89F95FFA88F8C145B0
:1098600029D25FFA89F919F804007D2820D15FFA1E
:1098700089F919EB0400407890F020005FFA89F92B
:1098800009F804005FFA88F85FFA89F9B8EB090073
:10989000821E92B25FFA89F919EB0400811C5FFA0B
:1098A00089F919EB0400401CFFF7F6FDB8F1010837
:1098B00019F10109CFE7B8F101095FFA89F9B9F1A6
:1098C0000A0F2CD35FFA89F9B9F1020189B2601C41
:1098D000FFF73DFF5FFA89F919EB040111F8011C4C
:1098E000C0B2814218D1607907000620C0B25FFA89
:1098F00089F9B9F1010188420ADAC0B2015D0E00AE
:10990000C0B2015D7940C0B201553700401CEDE79F
:1099100019F10100C0B203E0B9F10109CDE700205F
:10992000BDE8F28370B504000D0000262800C0B227
:10993000B6B280B2864210D2B6B2305D68280AD183
:10994000A91BC9B2B6B23019FFF76BFF002802D0CD
:10995000B6B2301902E0761CE8E7002070BD70B5A1
:1099600004000D00A07A10F10D06EDB2F6B2B5427A
:1099700001D2002018E02078682814D1F6B23019FE
:1099800010F8010C16280ED1F6B2B11E89B22000D3
:10999000FFF794FEF6B2311911F8021CC0B28842EA
:1099A00001D1012000E0002070BD70B504000D0061
:1099B0000026B6B2ADB2AE4210D2B6B2305D682863
:1099C0000AD1A91BC9B2B6B23019FFF7C8FF0028E7
:1099D00002D0B6B2301902E0761CEAE7002070BD72
:1099E000407A0C30C0B2704770B504000D00607A48
:1099F00010F10C06EDB2F6B2B54201D200201AE029
:109A00002078682816D1E079682813D1607A001987
:109A1000C07A16280ED1F6B2B11E89B22000FFF727
:109A20004DFEF6B2311911F8021CC0B2884201D1C4
:109A3000012000E0002070BD70B504000D0000267C
:109A4000B6B2ADB2AE4210D2B6B2305D68280AD11D
:109A5000A91BC9B2B6B23019FFF7C6FF002802D061
:109A6000B6B2301902E0761CEAE7002070BD38B5C6
:109A700004000D00ADB2052D01DA00200DE02078C4
:109A8000682809D10321601CFFF718FE2179C0B2B4
:109A9000814201D1012000E0002032BD70B50400F8
:109AA0000D000026B6B2ADB2AE4210D2B6B2305DF5
:109AB00068280AD1A91B89B2B6B23019FFF7D7FFBF
:109AC000002802D0B6B2301902E0761CEAE7002086
:109AD00070BD2DE9F04104000D0016001F00B046D6
:109AE000682088F80000102088F801000722210073
:109AF00018F10200FFF7D0FC012088F809000320CC
:109B000088F80A00EDB2002D01D0902000E01F205F
:109B100088F80B00EDB2002D01D01F2000E090204E
:109B200088F80C00002088F80D0098F80A0010F161
:109B30000B0189B24046FFF7C1FD88F80E001620E0
:109B400088F80F0098F80A000D303880BDE8F081E1
:109B50002DE9FC4104000D0016002F000721200014
:109B6000FFF766FD80460020C0B2072807DAC0B2C2
:109B7000211A897900AAC0B28154401CF4E74046FA
:109B800002F03CFE6820387000207870FA20B8702F
:109B9000FA20F8701020387102F040FEFF2190FB8F
:109BA000F1F201FB1200401C78712E20B8710020E8
:109BB000F8710420387204220DF1030117F1090035
:109BC000FFF76AFC002078731620B8730F21380065
:109BD000FFF7D1FD0C21781CFFF7B9FD78730F2139
:109BE0003800FFF7DCFD3080BDE8F381F8B50400F4
:109BF0000D00160068202870802068700622FF2162
:109C0000A81CFFF759FC0C2028720C206872002059
:109C1000A8727020E872202028730C20687301203D
:109C2000A8730522210015F10F00FFF735FCFF2076
:109C30002875FF206875FF20A87517212800FFF7F9
:109C400014FD0700EF75BFB2380A28761620687633
:109C50001A203080F1BDF0B583B004000D0016006D
:109C60002F000020C0B2072807DAC0B2211A897974
:109C700000AAC0B28154401CF4E7EB203870802069
:109C8000787004220DF10301B81CFFF705FC0020D9
:109C9000B87107213800FFF711FDF87108203080F6
:109CA000F7BD70B504000D0016006820287006226C
:109CB0002100681CFFF7F0FB6820E8710120287282
:109CC000022068724320A872C320E872687A10F1FB
:109CD0000A0189B22800FFF7F1FC28731620687387
:109CE000687A0C30308070BD70B504000D0016002D
:109CF0006820287006222100681CFFF7CDFB682031
:109D0000E87101202872022068724320A872C320E3
:109D1000E8720C212800FFF7D1FC28731620687325
:109D20000E20308070BD70472DE9F84304000D000F
:109D300016001F00DDF82080290089B22000FFF7FF
:109D400034FE8146B9F1000F01D1002033E0072233
:109D500019F102013000FFF7C3FC002801D10020F7
:109D600029E099F8090010F0C000C02801D10020B6
:109D700021E00222AE4919F10B00FFF7B1FC0028E7
:109D800009D10222AB4919F10B00FFF7A9FC002809
:109D900001D100200FE099F812003870042219F167
:109DA0000E01781CFFF778FB022219F11F014046D3
:109DB000FFF772FB0120BDE8F2832DE9F0410400BA
:109DC0000D0016001F00DDF818802900C9B2200020
:109DD000FFF7A8FD0100002901D100202DE08879BE
:109DE000AE2801D0002028E00020C0B204280BDA01
:109DF000C0B24218527AC0B2331ADB789A4201D00C
:109E000000201AE0401CF0E72C2038700020787009
:109E1000487CB870087CF870C87B3871487B1F227A
:109E2000104201D0032002E0487BC0F3401088F8C4
:109E30000000012088F801000120BDE8F0812DE933
:109E4000F84304000D0016001F00DDF82080A14635
:109E500000A879490A68026099F808008C2801D0A6
:109E6000002022E00522310019F10F00FFF738FC35
:109E7000002801D1002018E0042200A919F11900DE
:109E8000FFF72EFC002801D000200EE02C203870B7
:109E9000042219F11901781CFFF7FEFA022219F1C8
:109EA0001D014046FFF7F8FA0120BDE8F2832DE9D5
:109EB000F84304000D0016001F00DDF82080A146C5
:109EC00099F806000F2801D0002035E099F801002C
:109ED000902801D000202FE016214846FFF7EEFB26
:109EE00099F81610C0B2814201D0002024E0002071
:109EF000C0B204280CDAC0B210EB09018978C0B2F4
:109F0000321AD278914201D0002015E0401CEFE7D0
:109F10002C20387099F80800787099F80900B8700A
:109F200099F80A00F87000203871002088F80000C5
:109F3000002088F801000120BDE8F2832DE9F041FE
:109F400004000D0016001F00DDF81880290089B2FA
:109F50002000FFF7A3FD0100002917D02C20387046
:109F6000002078704878B8708878F870C87810F059
:109F70000F003871C878C0B2800810F0010088F86E
:109F80000000012088F80100012000E00020BDE869
:109F9000F0812DE9F84304000D0016001F00DDF8E4
:109FA0002080A14625480088ADF8000099F80800F7
:109FB000812801D0002039E099F80900062801D055
:109FC000002033E00622310019F10100FFF788FB81
:109FD000002801D1002029E0002099F80910C0B222
:109FE00088420AD2C0B210EB0901897A3339C0B273
:109FF00010EB09029172401CEFE7022200A919F14F
:10A000000A00FFF76DFB002801D100200EE02C2094
:10A010003870042219F10C01781CFFF73DFA00207A
:10A0200088F80000002088F801000120BDE8F283D4
:10A030005C0500205E05002040FF00080295000836
:10A04000C0B2DFF8EC11086070470021764A126850
:10A050001100890889000143734A1160704770B488
:10A0600000210022002300246F4D2D6815F00C05FF
:10A0700029000D00002D04D0042D05D0082D06D098
:10A0800026E06D4D056025E06C4D056022E0664DD3
:10A090002D6815F470152A00634D2D6815F4803570
:10A0A0002B00920C921C002B04D1654D05FB02F590
:10A0B00005600CE05C4D2D68AD0304D55E4D05FBDD
:10A0C00002F5056003E05D4D05FB02F5056001E06A
:10A0D000594D0560544D2D6815F0F005290009090A
:10A0E000584D4D5D2C0005682E00E64046604E4DF3
:10A0F0002D6815F4E0652900090A524D4D5D2C00CC
:10A1000045682E00E6408660474D2D6815F4605581
:10A110002900C90A4B4D4D5D2C0045682E00E640D4
:10A12000C660414D2D6815F440452900890B464D08
:10A130004D5D2C00C568B5FBF4F5056170BC70473A
:10A14000C9B2002905D0414A126802433F4B1A6048
:10A1500004E03E4A126882433C4B1A607047C9B221
:10A16000002905D03A4A12680243394B1A6004E0CC
:10A17000374A12688243364B1A607047C9B20029C9
:10A1800005D0344A12680243324B1A6004E0314A67
:10A19000126882432F4B1A607047C0B22E49086084
:10A1A000704710B40100002200230020C9B24C09FE
:10A1B000E4B22200012A03D11A4C2468230008E0EB
:10A1C000022A03D11B4C2468230002E0234C24689C
:10A1D0002300C9B211F01F0422001C00D440E40780
:10A1E00002D50124200001E000242000C0B210BCF0
:10A1F00070471A48006850F080701849086070472E
:10A2000001000020094A1268C9B20A4202D00122A4
:10A21000100001E000221000C0B270471049087021
:10A220007047000000100240041002400810024075
:10A23000600042422010024000127A000024F40024
:10A2400000093D00C0040020440500201410024015
:10A25000181002401C1002404C00424224100240E0
:10A260000A100240DFF8E00300887047DFF8D813D7
:10A27000088070471CB504004AF6BB20ADF800000A
:10A28000A4B2312C02DAADF8024002E03020ADF881
:10A290000200042100A8FFF7CBF9ADF80400BDF8D7
:10A2A0000200FFF7E3FF062200A9002000F04EFCA9
:10A2B00013BD00B583B0062200A9002000F0B9FC50
:10A2C000042100A8FFF7B4F9BDF8041080B2814260
:10A2D00005D1BDF80200DFF87013088002E00C2001
:10A2E000FFF7C8FFDFF8600300880EBD002080B2D2
:10A2F000C82811DADFF8541380B2182202FB0011CB
:10A300000979002906D1DFF8441380B2182202FB34
:10A31000001002E0401CEAE70020704738B5040056
:10A32000DFF82C0300680500002D0BD00722210068
:10A3300015F10800FFF7D4F9002801D0280002E049
:10A340002D68F1E7002032BDDFF804030068002823
:10A3500001D1012050E0DFF8F8020068007C0228FB
:10A360000DD10020DFF8E82212681071DFF8E0025A
:10A3700000680068DFF8D822106001203CE0DFF8B8
:10A38000D0020068010000290DD00868007C022876
:10A3900007D100200A681071086800680860012071
:10A3A0002AE00968EFE7DFF8A8020068007C0028CF
:10A3B0000DD10020DFF8982212681071DFF89002AA
:10A3C00000680068DFF888221060012014E0DFF8E0
:10A3D00080020068010000290DD00868007C002878
:10A3E00007D100200A681071086800680860012021
:10A3F00002E00968EFE7002070470FB410B5DFF8FE
:10A40000500200680400002C0FD0072204A914F1A8
:10A410000800FFF765F9002805D0DFF83802FCF7DF
:10A42000B0FF200027E02468EDE7FFF75FFF04009E
:10A43000002C11D1FFF788FF002807D0FFF756FF47
:10A440000400DFF81402FCF79CFF05E0DFF80C02C3
:10A45000FCF797FF00200EE0182202A92000FFF76A
:10A460001BF801202071DFF8E80100682060DFF8A8
:10A47000E0010460200010BC5DF814FB30B589B029
:10A4800004002000FFF74AFF0500002D05D0012041
:10A4900028710020E873280016E001208DF80C00D8
:10A4A00000208DF8180000208DF8170007222100E9
:10A4B00004A8FEF7F1FF02A984B06846182200F054
:10A4C00011FC0FBCFFF799FF09B030BD38B504008F
:10A4D0000D0010222900A4B2200110F5807080B276
:10A4E00000F0A7FB002809D00E212800FFF7A0F8F4
:10A4F000E98980B2884201D1012000E0002032BD0C
:10A5000080B5042200A9802000F093FB00280BD026
:10A51000022100A8FFF78CF8BDF8021080B281423A
:10A5200002D1BDF8000000E0002002BD10B582B0ED
:10A530000400ADF80040022100A8FFF779F8ADF85B
:10A540000200042200A9802000F000FB13BD10B51A
:10A5500082B00020FFF7EAFF4FF6FF70ADF8000071
:10A560000024A4B2C82C0ADA022200A9A4B2200155
:10A5700010F5807080B200F0E9FA641CF1E713BDB9
:10A580007FB5FFF7BDFF04000025A4B2C92C03DB93
:10A590003348FCF7F6FE2EE0A4B2002C03D131487C
:10A5A000FCF7EFFE27E026A0FCF7EBFE0026B6B294
:10A5B000C82E20DA00A9300080B2FFF787FF0028FC
:10A5C00017D0BDF8000048F69901884211D16D1CE2
:10A5D000B6B231002448FCF7D4FE1AA0FCF7D1FE35
:10A5E00007210DF10700FCF771FFADB2A4B2A5423F
:10A5F00001D2761CDBE77FBD10B515480068002846
:10A6000002D11A48FCF7BDFE0DA0FCF7BAFE1048B7
:10A6100000680400002C11D021791548FCF7B1FE28
:10A6200061791448FCF7ADFE06A0FCF7AAFE0721ED
:10A6300014F10800FCF74AFF2468EBE710BD0000A6
:10A640000D0A000069643A0060050020645500208E
:10A65000E4860020B8FB0008D0FB000848FD000895
:10A66000ACFA000858FD0008A0FE000868FD0008CC
:10A67000ACFE0008B8FE000828490143284A1160D2
:10A68000704770B4002400220F23C178002922D023
:10A690002349096811F4E061D1F5E061090A0C0071
:10A6A000D4F104010A0019000B00E3404178914005
:10A6B0000C00817819400C4324011A4905786C5428
:10A6C0000121057815F01F05A940174D0678761170
:10A6D00045F8261009E00121057815F01F05A9406D
:10A6E000124D0678761145F8261070BC7047104A56
:10A6F0000A4002430F4B1A607047042806D10E49E6
:10A70000096851F004010C4A116005E00A49096822
:10A7100031F00401084A1160704700000000FA059A
:10A720000CED00E000E400E000E100E080E100E08A
:10A7300080FFFF1F08ED00E010E000E010B582B0E0
:10A74000040003208DF802008020ADF80000E4B280
:10A75000012C03D104208DF8030002E014208DF8B1
:10A76000030000A9DFF8D803FCF7DEFC03208DF816
:10A7700002004020ADF8000010208DF8030000A971
:10A78000DFF8BC03FCF7D0FC13BD00221100C9B2F6
:10A79000C0B2814201D2491CF9E7704780B501215E
:10A7A0000820FFF7DCFC0121DFF89803FCF777FDB8
:10A7B00003208DF802008020ADF8000014208DF8F1
:10A7C000030000A9DFF87803FCF7AEFC03208DF846
:10A7D00002004020ADF8000010208DF8030000A911
:10A7E000DFF85C03FCF7A0FC01BD80B58021DFF839
:10A7F0005003FCF74EFD4021DFF84403FCF749FD10
:10A800000220FFF7C2FF8021DFF83403FCF744FD8C
:10A810000220FFF7BAFF4021DFF82403FCF73CFDDC
:10A820000220FFF7B2FF01BD80B58021DFF81003E1
:10A83000FCF732FD0220FFF7A8FF4021DFF80003FC
:10A84000FCF727FD8021DFF8F802FCF725FD022048
:10A85000FFF79BFF8021DFF8E802FCF71AFD01BD3E
:10A8600010B500240120FFF769FF4021B448FCF730
:10A8700010FD0120FFF789FF8021B148FCF7EFFCB4
:10A88000012802D10020040001E001200400402141
:10A89000AB48FCF701FD0120FFF777FF0020FFF731
:10A8A0004DFF2000C0B210BD80B58021A448FCF748
:10A8B000F3FC0120FFF769FF4021A148FCF7ECFC05
:10A8C0000120FFF762FF40219D48FCF7E2FC0120D8
:10A8D000FFF75BFF40219A48FCF7DEFC8021984897
:10A8E000FCF7D7FC01BD80B580219548FCF7D1FC71
:10A8F0000120FFF74AFF40219148FCF7CDFC0120E1
:10A90000FFF743FF40218E48FCF7C3FC0120FFF70F
:10A910003CFF40218A48FCF7BFFC01BD38B504006C
:10A9200040218748FCF7B8FC00200500EDB2082D57
:10A930001CDAE4B2200604D580218148FCF7A9FC8A
:10A9400003E080217E48FCF7A7FC40217C48FCF70F
:10A95000A0FC0120FFF719FF40217948FCF79CFC7F
:10A960000120FFF712FF64006D1CDFE75A20FFF79C
:10A970000CFF31BD38B500250120FFF7DFFE402177
:10A980006F48FCF789FC0120FFF7FFFE0020040060
:10A99000E4B2082C1BDA6D0040216948FCF779FC11
:10A9A0000120FFF7F2FE80216548FCF758FC0128E2
:10A9B00002D155F0010501E015F0FE054021604887
:10A9C000FCF76AFC0120FFF7E0FE641CE0E70020D2
:10A9D000FFF7B4FE2800C0B232BD80B5FFF705FF17
:10A9E000A020FFF79BFFFFF73BFF012803D1FFF7F4
:10A9F0001BFF012002E0FFF717FF002002BD80B51A
:10AA0000FDF796F950490968C91C8842F8D3FFF749
:10AA1000E4FF0028FBD001BD2DE9F04104000D004A
:10AA2000002600275FF0000820000700A4B2200ADB
:10AA30008046FFF7E4FFFFF7D8FEA020FFF76EFF88
:10AA4000FFF70EFF002801D100202CE04046C0B2E5
:10AA5000FFF764FFFFF704FF002801D1002022E088
:10AA60003800C0B2FFF75AFFFFF7FAFE002801D105
:10AA7000002018E0A1200600FFF7B7FE3000C0B2AA
:10AA8000FFF74CFFFFF7ECFE002801D100200AE0A1
:10AA9000FFF770FF2870FFF726FF0120FFF775FE14
:10AAA000FFF7C2FE0120BDE8F0812DE9F843040064
:10AAB0000D00160020000700A4B2200A8046FFF710
:10AAC0009EFFFFF792FEA020FFF728FFFFF7C8FECA
:10AAD000002801D1002030E04046C0B2FFF71EFF41
:10AAE000FFF7BEFE002801D1002026E03800C0B2EA
:10AAF000FFF714FFFFF7B4FE002801D100201CE08F
:10AB00005FF000095FFA89F9F6B2B1450ED25FFA3B
:10AB100089F919F80500FFF701FFFFF7A1FE0028EA
:10AB200001D1002009E019F10109EBE7FFF77CFEF4
:10AB3000FDF7FEF8044908600120BDE8F28300003B
:10AB4000000C014000023000C08600202DE9F84FC3
:10AB500004000D001600FFF721FEA146A4B28020DC
:10AB600094FBF0F101FB1041D1F18007AA46B046F9
:10AB70003800C0B280B2B6B2B0424CD23A00D2B2C3
:10AB80005146484680B2FFF790FF002801D10020CF
:10AB90004DE0FFB217EB0909FFB217EB0A0AFFB24B
:10ABA000F01B80461FFA88F8802098FBF0F0ADF883
:10ABB00002001FFA88F8802098FBF0F101FB108159
:10ABC000ADF800105FF0000BBDF802001FFA8BFB20
:10ABD000834510D280225146484680B2FFF765FF78
:10ABE000002801D1002022E019F180091AF1800A21
:10ABF0001BF1010BE8E7BDF80000002816D0BDF8F6
:10AC00000020D2B25146484680B2FFF74EFF0028DE
:10AC10000CD100200BE03200D2B22900200080B21B
:10AC2000FFF743FF002801D1002000E00120BDE82C
:10AC3000F28F2DE9F04104000D001600B6B2002E8F
:10AC400001D100203CE0FFF7DAFEFFF7A7FD290065
:10AC5000200080B2FFF7E0FE002801D100202FE0A5
:10AC6000761EB6B2002E2AD0A1200700FFF7BDFD48
:10AC70003800C0B2FFF752FEFFF7F2FD002801D105
:10AC800000201DE05FF000081FFA88F8B6B2B0455A
:10AC900011D2FFF76FFE1FFA88F818EB0501487014
:10ACA0001FFA88F8B6B2701E804501DAFFF7FCFD86
:10ACB00018F10108E8E7FFF716FEFFF7B5FD0120E0
:10ACC000BDE8F08162B38B0708D0521E11F8013B3A
:10ACD00000F8013B00F024808B07F6D1830740F099
:10ACE000208000BF103A07D330B4B1E83810103AD2
:10ACF000A0E83810F9D230BC530724BFB1E80810DF
:10AD0000A0E8081044BF51F8043B40F8043BD207C8
:10AD100024BF31F8022B20F8022B44BF0B780370BC
:10AD20007047083A07D3B1E80810083A40F8043BE6
:10AD300040F804CBF7D25307E4E7000007B582B030
:10AD400001210498FFF70BFABDF80800ADF80000E8
:10AD500010208DF8030002208DF8020000A903984E
:10AD6000FCF7E2F902A807C800F02FF805B000BD13
:10AD700080B50C4807C8FFF7E1FF0B4807C8FFF78D
:10AD8000DDFF0A4807C8FFF7D9FF094807C8FFF7E2
:10AD9000D5FF084807C8FFF7D1FF074807C8FFF7E6
:10ADA000CDFF01BDE0040020EC040020F8040020E9
:10ADB00004050020100500201C05002007B4BDF884
:10ADC00000000199486103B0704707B4BDF8000066
:10ADD0000199086103B07047F0B587B00400002501
:10ADE000002600A801F0EAFC002801D1002040E084
:10ADF0000C2203A900A802F071FA0027BFB2B7F530
:10AE0000806F0ADA01F00AFDFF2190FBF1F201FBED
:10AE10001200BFB238557F1CF0E70020B0F5806FFC
:10AE200010D22021B0FBF1F202FB1102002A07D15F
:10AE300003A9F6B2715C0155761CF6B2102E01DA48
:10AE4000401CEBE740F2FE312000FEF7F1FB05006D
:10AE5000ADB24FF4807095FBF0F101FB105184F816
:10AE6000FE13ADB24FF4807095FBF0F084F8FF0351
:10AE7000012007B0F0BD00B5ADF2044D0020B0F5E3
:10AE8000806F08D24549095CC9B2FF2901D0002072
:10AE900018E0401CF3E700A8FFF79EFF002810D041
:10AEA0003E4801F0F1FB002809D14FF4806200A96F
:10AEB0003A4801F006FC002801D1012002E0002000
:10AEC00000E000200DF2044D00BD2DE9F0418CB0F2
:10AED00000254FF6FF7600275FF0010800A801F07B
:10AEE0006DFC002806D00C2207A900A802F0F6F994
:10AEF000002001E000204EE080B240F2FE318842A6
:10AF000024DA80B22549095C0C00E4B2FF2C01D0A0
:10AF100000218846B6B22249320092B2E4B26240C1
:10AF2000D2B231F8121091EA162680B2202190FB9D
:10AF3000F1F202FB1102002A06D1EDB2102D03D26C
:10AF400003A9EDB26C546D1C401CD5E786F47F4616
:10AF500096F0FF0613480078C0B213490978C9B2C9
:10AF60004FF4807202FB010007005FFA88F8B8F125
:10AF7000010F02D1FFF77FFF0DE0BFB2B6B2B742BB
:10AF800008D1102207A903A8FEF7AAFB002801D0C8
:10AF9000012000E000200CB0BDE8F081003800087E
:10AFA000D8F20008FE3B0008FF3B0008C0B20328AF
:10AFB00002DADFF8A01808707047DFF89808007808
:10AFC000704730B480B2082190FBF1F1DFF8882897
:10AFD000891880B2082290FBF2F2DFF87C38D21890
:10AFE000527B012380B2082490FBF4F505FB140585
:10AFF000AB401A434A7330BC704710B4010089B2A9
:10B00000082091FBF0F0DFF850288018407B0122E7
:10B0100089B2082391FBF3F404FB1314A2401042FD
:10B0200001D0012000E0002010BC704738B50400BA
:10B030000025ADB2A4B2A54209D2280080B2FFF724
:10B04000DCFF002801D1002002E06D1CF1E70120A7
:10B0500032BDF0B401004FF6FF768C1EDFF8FC57CE
:10B06000032901D200202CE02000441E00280FD02C
:10B07000287803006D1CB6B2DFF8E4073700BFB2D2
:10B08000DBB25F40FFB230F8170090EA1626EBE71C
:10B0900086F47F4696F0FF06287803006D1CDBB22D
:10B0A0004FF4807000FB03F00200287803006D1C51
:10B0B000DBB29A18B6B292B2964201D1012000E0FA
:10B0C0000020F0BC7047F0B5A1B004000D001600E0
:10B0D000A4B28020DFF8841700FB0417F6B2320018
:10B0E00092B2290000A8FEF7D7F972B6F6B2320084
:10B0F00092B22900380001F0E4FA62B621B0F0BD46
:10B1000010B504008C212000FEF792FAA4F88C0000
:10B11000DFF8500701F0B8FA002805D18E2221008F
:10B12000DFF8400701F0CDFA10BD80B58E22002176
:10B13000DFF82407FEF7DAF9DFF81C07FFF7E0FF76
:10B1400001BDF8B504000D0016001F006820DFF8EF
:10B15000181708701320DFF81017A1F8010056F037
:10B16000C000DFF80417C870DFF8FC06007910F0A3
:10B17000FE00DFF8F4160871DFF8EC06007910F035
:10B18000FD00DFF8E4160871DFF8DC06007910F046
:10B19000FB00DFF8D4160871DFF8CC06007910F058
:10B1A000F700DFF8C4160871DFF8BC06007910F06C
:10B1B0000F00DFF8B41608710020DFF8AC164871F4
:10B1C0000020DFF8A41688710020DFF89C16C871F3
:10B1D0000020DFF894160872DFF88C064472152000
:10B1E000DFF8841688720120DFF87C16C872002010
:10B1F000DFF874160873DFF87006C0F80D500E21E2
:10B20000DFF86806FEF75AFADFF85C164874162075
:10B21000DFF854168874FFB2022F05D11321DFF82E
:10B220004806FCF78FF804E01321DFF83C06FAF734
:10B2300070F8F1BD10B4020000230020C0B208284D
:10B2400007DAD2B21400044114F00104E318401CE0
:10B25000F4E79BB2012B01D0FF200FE00020030098
:10B26000D2B25208D2B2002A06D1C9B289B213EBC7
:10B27000C100F13080B201E05B1CF1E710BC704707
:10B28000F8B504000D0016001F0068202070EDB214
:10B29000A4F8015057F08000E070207910F0FE0013
:10B2A0002071207910F0FD002071207966F3820072
:10B2B0002071207910F0F7002071207910F00F0034
:10B2C000207104220021601DFEF7F6F8DFF8A005CA
:10B2D00000786072F1BD2DE9F04104000D000026F8
:10B2E0000A222100DFF88C050068FEF7F1F8DFF88C
:10B2F00088054078DFF8801589784FF4807202FB6A
:10B3000001081FFA88F818EB040010F8020CDFF8A7
:10B310006415096848771FFA88F818EB040010F8DC
:10B32000010CDFF850150968887714F10A0006004F
:10B33000DFF840050068407ADFF834150870DFF860
:10B34000340500680079C0F38000C0B200282DD019
:10B35000DFF820050068C0F80A60B61DDFF81405A4
:10B360000068D0F80A00FEF7CDF8002800F0B080A1
:10B37000DFF8000500680079C0B20009C0B20028FB
:10B380000ED0DFF8F0040068C0F80E60DFF8E404C7
:10B3900000680079C0B20009C0B2062101FB006656
:10B3A000DFF8D0040068C0F81260B61D3078DFF80E
:10B3B000C414096888757078DFF8B8140968C8750E
:10B3C000B078DFF8B01409680876F61CDFF8A4043A
:10B3D0000068017EDFF89C040068C07DFFF72AFF4B
:10B3E0000700DFF890040068C0F81960DFF88404F3
:10B3F00000680079C0F38000C0B2002868D1DFF88F
:10B4000074040068807D032802D0152836D05FE0E0
:10B41000BFB2F12F31D1EDB2012D2ED1DFF854049E
:10B420000068C37800221721DFF85004FFF728FFD7
:10B430000320DFF8481488720120DFF84014C87236
:10B440000020DFF83814087301F05CFF09220100C6
:10B45000DFF82C04FEF720F81221DFF82804FEF7AD
:10B460002DF9DFF8181448751620DFF810148875C8
:10B470001721DFF80804F9F74CFF29E0BFB2F12FDC
:10B4800025D1FFF79AFD002810D12800C0B2FFF7A0
:10B490008DFD00230A22DFF8DC030068D0F81910C4
:10B4A000DFF8E4030068FDF7C0FB10E0FFF785FD5F
:10B4B000EDB2A8420BD100230A22DFF8B8030068DE
:10B4C000D0F81910DFF8C0030068FDF7AEFBFFE706
:10B4D000BDE8F08138B504006078A1784FF480723F
:10B4E00002FB01052078682814D1EDB2281910F864
:10B4F000010C16280ED1EDB2691F89B2E01CFEF7CF
:10B50000DDF8EDB2291911F8021CC0B2814201D157
:10B51000012000E0002032BD0100CA0A10004FF4F3
:10B520000062B1FBF2F303FB1213002B00D0401CAE
:10B5300080B2704770B504002000FFF7EDFF0500F2
:10B540000026ADB2AE4227D24FF400624FF4006045
:10B55000C24900FB0611DFF83403FDF7B9FF4FF4D1
:10B56000006000FB06F010F1006001F08DF800288B
:10B5700010D14FF40062C5494FF4006000FB06F0A3
:10B5800010F1006001F09DF8002801D0002004E0D7
:10B59000761CD6E7002000E0012070BD38B504001D
:10B5A0000D00D4F8050080B2FFF727FD002804D075
:10B5B000B748FBF7E6FE002053E0D4F80510B54885
:10B5C000FBF7DFFEB4F80920D2B2D4F80B10D4F8A0
:10B5D000050080B2FFF777FDD4F8050080B2FFF7D1
:10B5E000F0FC6889401C6881D4F805002881D4F8F3
:10B5F0000500B4F80310491E884231D1E888FFF7EE
:10B6000015FD012825D1A448FBF7BBFE2968A348F6
:10B61000FBF7B7FEB4F80300401E8021B4F8092000
:10B6200001FB002028602078032806D1022028731F
:10B630002800FFF765FD012013E02078FD2801D1E7
:10B6400001200EE0FFF771FD9548FBF79AFE002000
:10B6500007E0FFF76AFD9348FBF793FE002000E048
:10B66000002032BD10B500243B2C08D24FF40060FE
:10B670007A4900FB041001F007F8641CF4E710BDE0
:10B6800010B504000022FF210120FDF765FA7E4974
:10B69000086000235FF0FF3283497B480068FDF7B4
:10B6A0009FFC0B2280498148FDF712FF80487F49AB
:10B6B000C1F80B007D48D0F805000028E9D17D488D
:10B6C000FBF75FFEFBF734FE8E2200216248FDF798
:10B6D0000DFFFFF7C7FF4FF4FA70FCF749FA01209E
:10B6E0005D4908737148B0F803005B49C8805A4847
:10B6F000C1887148FBF745FE002070490860564933
:10B700006A48FFF74BFF6E490870524803780A22D7
:10B710006648D0F8051056480078FFF712FD4D48EE
:10B720000078012806D13220FCF722FA4FF461405C
:10B73000F9F7FAFD002340F2DC525B4952480068F9
:10B74000FDF74EFC012869D10B2257495748FDF7F8
:10B75000BFFE57485549C1F80B005448D0F80500C2
:10B7600056490968491C88420CD0FFF7DEFCFBF7FC
:10B77000E4FD38480078012803D14FF41650F9F75A
:10B78000D3FD86E74D480068401C4C4908603249AB
:10B790004648FFF703FF4A4908702E4803780A22FB
:10B7A0004248D0F8051032480078FFF7CAFC4448F8
:10B7B00000780028BED00020414908703B4800783E
:10B7C000032805D19620FCF7D3F9FDF79DFFB1E7DB
:10B7D00036480078FD2816D11F480068FFF739FC6D
:10B7E0000028A7D01C480068FFF7A4FE002801D15C
:10B7F000FDF78AFF1748007801289BD14FF41650B7
:10B80000F9F792FD96E713480078012803D14FF429
:10B810001650F9F789FDFFF788FC8BE70D48007893
:10B82000012803D14FF41650F9F77EFD8E22002136
:10B830000948FDF75BFE2CE700B583B000200190BE
:10B84000032000900023C82200211E48FCF712F8B4
:10B8500007BD000071870020F88200200028020840
:10B86000D8F2000800400008948600209786002047
:10B870007087002054050020A4850020DC8500206E
:10B88000E9850020DF8500205887002024680020FB
:10B89000E0FC00081CFB000800FC000838FB000866
:10B8A00054FA0008F4FC0008F8810020A886002063
:10B8B0000382002008FE000854FB00085C8700207B
:10B8C0007287002081B6000808B584B00023029377
:10B8D00011B90093019302E00090481E019004AB5F
:10B8E00000A907487844183001F056FD009911B1BD
:10B8F000009A00211170002858BF029805B000BDC1
:10B900000FB8FFFF001F5FF080730360001F4B083C
:10B910005B000360001F0FF20D0303601438026028
:10B920002038704780B56548006810F1010F03D0DA
:10B930006349EE2000F048FE102080F31188BFF329
:10B940004F8FBFF36F8FFEE700B583B05D4801787E
:10B950000191FF21017001788DF800109DF8001011
:10B9600011F01001584A11700721584A11609DF8D2
:10B97000001009060AD555490968491E534A116045
:10B980009DF8001049008DF80010F0E74F49096854
:10B9900009024E4A11604D49096811F4E0614B4AB1
:10B9A0001160019901704A48006850F470004849DC
:10B9B00008604748006850F070404549086000F052
:10B9C0004DF800203D49086002F0F1FB00200EBD5B
:10B9D00080B5102080F31188BFF34F8FBFF36F8FB6
:10B9E00036480068401C3549086034480068012822
:10B9F00008D138480068000604D031494FF4A670D9
:10BA000000F0E2FD01BD80B52C480068002804D19B
:10BA10002B4940F2531000F0D7FD28480068401E23
:10BA20002649086025480068002802D1002080F3DC
:10BA3000118801BD80B5102080F31188BFF34F8FAE
:10BA4000BFF36F8FFCF779F9002803D05FF08050C7
:10BA500020490860002080F3118801BD1E4800685D
:10BA6000C0084FF4FA71B0FBF1F0401E1B490860AA
:10BA700003201B490860704738B5EFF305800400C8
:10BA8000102C0DD317480068205C05000E48007884
:10BA9000EDB2854204D20A4940F2472000F094FDFD
:10BAA0000A4800681049096811F4E061884204D22C
:10BAB000034940F2572000F087FD31BD40050020CA
:10BAC000E4F7000800E400E06D870020E086002035
:10BAD00020ED00E004ED00E04805002014E000E067
:10BAE00010E000E03CFF00080CED00E080B5FBF743
:10BAF00043FC002805D000F020F8A6A0FBF741FC8D
:10BB000003E0DFF8B006FBF73CFC01BD01000020BC
:10BB1000C0B2FF280FD0C0B2425C202A07D0C0B20A
:10BB2000425C0D2A03D0C0B2425C0A2A01D1C0B2E5
:10BB300002E0401CECE7002070472DE9F8430024A8
:10BB4000002501275FF00009DFF86C0600785FFA36
:10BB500089F981455AD2DFF864065FFA89F90C2128
:10BB600001FB09000068060000200400DFF84C0615
:10BB70005FFA89F90C2101FB0900006800780500D3
:10BB8000EDB2002D0CD0641CDFF830065FFA89F9A5
:10BB90000C2101FB09000068E4B2205C0500EFE71E
:10BBA00001200700DFF81806FFF7B0FF80465FFAB4
:10BBB00088F8E4B2A04502D00020070023E000206E
:10BBC000C0B2E4B2A0420CD2C0B2815DDFF8F02571
:10BBD000C0B2825C914202D00020070001E0401C0C
:10BBE000EEE7E4B2002C01D100200700FFB2002FE5
:10BBF00009D0DFF8C8055FFA89F90C2101FB0900BB
:10BC00004068804702E019F101099DE7FFB2002F6B
:10BC100011D1DFF8AC0500780D2809D0DFF8A005B8
:10BC200000780A2804D0DFF89C05FBF7AAFB02E0A5
:10BC30008CA0FBF7A6FBBDE8F1830100C9B2302957
:10BC400006DBC9B23A2903DAB1F13000C0B214E020
:10BC5000C9B2612906DBC9B2672903DAB1F157001D
:10BC6000C0B20AE0C9B2412906DBC9B2472903DAEA
:10BC7000B1F13700C0B200E0002070472DE9F04775
:10BC800004000D0000260027FBF776FBBFB28742B9
:10BC90007CD2DFF82C05BFB2385C202874D1761C2A
:10BCA000F6B2EDB2AE426FD1DFF81405BFB238186C
:10BCB000807820280DD0DFF80805BFB238188078CA
:10BCC0000D2806D0DFF8F804BFB2381880780A28AB
:10BCD00008D1DFF8EC04BFB238184078FFF7ADFFA9
:10BCE000207050E0DFF8D804BFB23818C0782028A0
:10BCF0000DD0DFF8CC04BFB23818C0780D2806D0BC
:10BD0000DFF8BC04BFB23818C0780A2817D1DFF8B2
:10BD1000B004BFB238184078FFF78FFF81460A2081
:10BD200000FB09F9DFF89804BFB238188078FFF7F4
:10BD300084FF804619EB080884F8008023E0DFF8D0
:10BD40008004BFB238184078FFF777FF8046642040
:10BD500000FB08F8DFF86804BFB238188078FFF7F6
:10BD60006CFF81460A2000FB09F9DFF85404BFB2DA
:10BD70003818C078FFF761FF824619EB080010EB16
:10BD80000A0A84F800A003E07F1C7DE700202070F1
:10BD9000BDE8F087433E00002DE9F84304000D00A4
:10BDA0005FF00009002627005FF00008FBF7E4FAC7
:10BDB0000100002080461FFA88F889B288454BD2DE
:10BDC000DFF8FC031FFA88F818F80000202840D19B
:10BDD00019F101095FFA89F9EDB2A94539D1DFF806
:10BDE000E0031FFA88F818EB00004078202801D003
:10BDF000012000E00020DFF8C8231FFA88F818EBC4
:10BE0000020252780D2A01D0012200E00022DFF860
:10BE1000B0331FFA88F818EB03035B780A2B01D0C4
:10BE2000012300E00023C0B2D2B21040DBB21842BE
:10BE30000CD0DFF88C031FFA88F818EB000040786C
:10BE400038707F1C18F10108761CC8E73000C0B2BA
:10BE500004E018F10108AEE73000C0B2BDE8F2839B
:10BE6000000000000D0A000010B50400200002F0E0
:10BE7000AFF921002278302A04D16278782A01D1E2
:10BE8000801E891C002292B280B282421BD292B2E2
:10BE9000535C302B03DB92B2535C3A2B11DB92B232
:10BEA000535C612B03DB92B2535C672B09DB92B2CC
:10BEB000535C412B03DB92B2535C472B01DB100038
:10BEC00001E0521CDFE780B210BDF8B5040000A805
:10BED000002101602000FFF7C7FF0500ADB202207E
:10BEE00095FBF0F101FB1051002904D1ADB2022005
:10BEF00095FBF0F604E0ADB2022095FBF0F0461C95
:10BF00002078302808D16078782805D12A0092B2AC
:10BF1000A11C2000FDF7C0FA0027BFB2B6B2B7429D
:10BF200026D2BFB2002F0FD1ADB2022095FBF0F1A7
:10BF300001FB1051012907D100208DF80000BFB28C
:10BF4000385D8DF801000AE0BFB214F817008DF8D3
:10BF50000000BFB214EB470040788DF801001022BA
:10BF6000002100A802F04FF9BFB238557F1CD4E77A
:10BF7000F1BD10B588B0012100A8FFF70DFF9DF8B5
:10BF80000000302833D19DF8010078282FD19DF88A
:10BF90000E0000282BD100A8FFF766FF0C2803D065
:10BFA0008948FBF7EEF925E000A8FFF78EFF00A80F
:10BFB000FDF7C7FA05A8FDF7F0FA002813D083486B
:10BFC000FBF7DFF90024E4B2062C08DA05A8E4B296
:10BFD000001B417975A0FBF7D4F9641CF3E774A04A
:10BFE000FBF7CFF906E07A48FBF7CBF902E0794896
:10BFF000FBF7C7F908B010BD1CB500A8FDF7CDFAD6
:10C000007248FBF7BEF90024E4B2062C08DA00A857
:10C01000E4B2001B41797048FBF7B3F9641CF3E705
:10C0200063A0FBF7AEF913BD00B593B00AA82021B9
:10C0300002F0ECF801210AA8FFF7AEFE0AA8FFF70C
:10C0400044FF08A8FDF7A9FA68208DF80000062231
:10C0500008A90DF10100FDF73BFA68208DF80700F3
:10C0600011208DF808000C208DF8090000208DF8B3
:10C070000A00FF208DF80B0001208DF80C00002035
:10C080008DF80D0008220AA90DF10E00FDF720FA27
:10C0900000209DF80910C0B288420AD200A9C0B29F
:10C0A0004118897A333100AAC0B282189172401CBB
:10C0B000EFE79DF8090010F10A0189B200A8FDF729
:10C0C000FDFA00A99DF8092051188872162000A9D0
:10C0D0009DF809205118C8729DF8090010F10C0153
:10C0E000C9B200A8F9F789F913B000BD00B585B051
:10C0F000012100A8FFF750FE00A8FFF7E6FE00A808
:10C10000FEF7BCF9FEF778FA05B000BD10B586B0B1
:10C11000012100A8FFF740FE00A8FFF7D6FE00A807
:10C12000FEF7FCF80400002C02D12C48FBF729F99B
:10C1300006B010BD80B5012100A8FFF79FFD9DF856
:10C140000000F9F761FF00F001F801BD80B5F9F7D3
:10C1500082FF002803D12248FBF713F902E02148AF
:10C16000FBF70FF901BD00B587B001A8142102F05B
:10C170004DF801210DF10200FFF780FD022101A819
:10C18000FFF70AFE01A8FFF7A0FE00AB164A0DF16B
:10C1900005019DF8020080B2F9F7DEFABDF8001043
:10C1A0001148F9F748F807B000BD00002558000015
:10C1B0000D0A000074FA000862050020B4F60008B9
:10C1C000F877002018FC000808FD000818FD00089A
:10C1D0002CFC000890FA000804FF0008A0FB0008EF
:10C1E00040FC000854FC0008888300202DE9F04141
:10C1F00004005FF00008FBF717FD8F480068002877
:10C2000001D100F0AFF88D480068044261D1002CE4
:10C2100011D08B480068041914F0070F0BD014F1EB
:10C22000080014F00701441A14F0070F03D08549E1
:10C23000BF2000F0C9F9002C4BD083480068A04211
:10C2400047D3824806008148006805006868A0421C
:10C2500005D22868002802D02E002D68F6E776481F
:10C260000068854235D030687549096808188046ED
:10C27000286830607248006840006968091B88427D
:10C2800010D26019070017F00700002803D06D498D
:10C29000EC2000F099F96868001B78606C60380049
:10C2A00000F097F8684800686968401A66490860B5
:10C2B0006548006866490968884203D26248006898
:10C2C0006349086068685D49096808436860002040
:10C2D0002860FBF7B1FCB8F1000F01D100F061F963
:10C2E00018F00700002804D056494FF4967000F06B
:10C2F0006BF94046BDE8F08170B504002600002CC3
:10C300002FD04F480068361A350068684B490968D5
:10C31000084204D14B494FF4A07000F055F9286849
:10C32000002804D0474940F2411000F04DF96868F8
:10C3300042490968084214D02868002811D1686869
:10C340003E49096888436860FBF76EFC3E48006818
:10C35000696808183C490860280000F03AF8FBF7C3
:10C360006BFC70BD30B44FF4A0433A4C220012F085
:10C37000070F05D0D21DD208D2009B1A354CE31806
:10C380001100324C21600024304D6C605C1822009A
:10C390002B4C2468121BD208D200274C22600024A8
:10C3A000254D2D686C600024234D2D682C600800FD
:10C3B000141A4460204C246804604468244D2C60A6
:10C3C0004468214D2C605FF000441C4D2C6030BC53
:10C3D000704710B41D4B1A001368834201D21268D3
:10C3E000FAE7110053685B18834204D1536844682C
:10C3F000E31853601000010043685B181468A342FF
:10C4000011D113680C4C2468A34208D04368146807
:10C410006468E318436013681B68036005E0064B1B
:10C420001B68036001E013680360824200D0106063
:10C4300010BC704700000000D0860020DC86002081
:10C4400038FF00089CF70008D4860020B88600203A
:10C45000D88600206405002062F30F2262F31F4299
:10C46000401810F0030308D0C91A1FD3DB0748BFD8
:10C4700000F8012D28BF20F8022D130030B4144617
:10C480001546103928BF20E93C00FAD8490728BFD3
:10C4900020E90C0048BF40F8042D890028BF20F88F
:10C4A000022D48BF00F8012D30BC7047C91818BFD5
:10C4B00000F8012DCB0728BF00F8012D70470000C0
:10C4C00010B5040094E80700FEF778FC4FF4FA700A
:10C4D000FBF74EFB94E80700FEF777FC4FF4FA7089
:10C4E000FBF746FBEEE710B504000A2001F091FED1
:10C4F00001F0C6FE4FF47A70FBF73AFBF8E700B59F
:10C5000083B00020C0B2FF2805D0411C154AC0B23C
:10C510008154401CF6E700F02FF800200190012024
:10C520000090114B462200211048FBF7A3F9002090
:10C530000190032000900023C82200210C48FBF743
:10C5400099F9002001900420009000234622002148
:10C550000848FBF78FF9FBF76DF8FFF76DF9FBF76C
:10C560002CFBFEE7F87900201C050020C1C4000860
:10C5700049650008E7C4000880B501F091FE01F0AC
:10C5800094FE01F0F7FE0420FEF7B7F84FF4407078
:10C59000FEF772F8FEF7ECFBFDF725F8FEF7FEF864
:10C5A00001BD102080F31188BFF34F8FBFF36F8F51
:10C5B000FEE77047102282F31188BFF34F8FBFF35D
:10C5C0006F8FFEE77047000038B504000D000020B3
:10C5D0000090FFF7FDF90098002802D100BF00BFCE
:10C5E000F9E7FFF710FA31BD10F1080141605FF083
:10C5F000FF31816010F10801C16010F10801016193
:10C6000000210160704700210161704742684A6063
:10C6100093688B60936859609160086103685B1C44
:10C620000360704710B40B6813F1010F02D1046965
:10C63000220008E010F10804220054682468A34294
:10C6400001D35268F9E754684C604C68A1608A6075
:10C65000516008610468641C046010BC70470100EC
:10C6600008698A684B689A604A688B685A604268B1
:10C670008A4201D18A68426000220A610268521E21
:10C68000026000687047000038B50400042501F01E
:10C69000F7FD01F04BFF342001F0B1FF200001F065
:10C6A00059FF0500EDB2042D07D0EDB22A0021009C
:10C6B0004F48FAF766FE012002E001F042FF002039
:10C6C00032BD2DE9F84F04000D0016005FF00008A0
:10C6D000B1465FF0040A01F029FF342001F08FFF1A
:10C6E0001FFA89F9022099FBF0F101FB10910F006C
:10C6F000FFB2002F01D0B9F10109002080461FFAD6
:10C7000088F81FFA89F9C84529D21FFA88F818EB6A
:10C71000050040781FFA88F818F8051051EA002142
:10C7200089B21FFA88F818EB040001F042FF824634
:10C730005FFA8AFABAF1040F0ED05FFA8AFACDF8DE
:10C7400000A01FFA88F84346B6B2320021002948FB
:10C75000FAF717FE02202FE018F10208CFE7FFB228
:10C76000002F26D0B6B2002E23D0B6B2701910F822
:10C77000010C50F47F408346594689B21FFA88F86D
:10C7800018EB040001F015FF82465FFA8AFABAF14D
:10C79000040F0ED05FFA8AFACDF800A01FFA88F8CD
:10C7A0004346B6B2320021001248FAF7EAFD0220F1
:10C7B00002E001F0C6FE0020BDE8F28F010000207B
:10C7C000C0B20C2806DAC0B20B4A125CC0B24254A6
:10C7D000401CF5E70020C0B20C2807DAC0B2425C6A
:10C7E000FF2A01D0012002E0401CF4E7002070473E
:10C7F0006CF8000850F70008E8F7FF1F10B5044672
:10C80000044801F03CFF00210170034801F037FFAC
:10C81000046010BD0002002004020020F8B5344F6F
:10C82000384601F02CFF0446381D01F028FF05466C
:10C8300007F1080001F023FF064607F10C0001F0A4
:10C840001EFF23782B492C4A002B40D12B6802FB7A
:10C8500003132B60082702FB03132B6002FB031357
:10C860002B6002FB03132B6002FB03132B6002FB04
:10C8700003132B6002FB03132B6002FB03132B60DB
:10C880000346D5F800C002FB0C1CC5F800C043F8F5
:10C8900004CB7F1ED5F800C002FB0C1CC5F800C0FD
:10C8A00043F804CBD5F800C002FB0C1CC5F800C04F
:10C8B00043F804CBD5F800C002FB0C1CC5F800C03F
:10C8C00043F804CBDDD1C36F3360012323702B68A1
:10C8D00002FB03112960317801F01F0150F821207B
:10C8E00032602A6840F82120306880008008F2BD5C
:10C8F000000200205FF36E3C0D661900002101600C
:10C9000000214160DFF8C0188160DFF8C018C16005
:10C91000DFF8BC180161DFF8BC18416170472DE9F0
:10C92000F84F05008A46160000275FF00008002433
:10C930002868C0F3C5008046D8F14000040028688C
:10C9400010EBC60028602868B0EBC60F02D26868FA
:10C95000401C6860686810EB56706860A6421ED381
:10C9600018EB050010F11809220051464846FEF761
:10C97000A9F915F1180115F1080000F07EF827005B
:10C9800017F14000864207D317EB0A0115F10800A2
:10C9900000F073F84037F3E70020804601E0002004
:10C9A0000700F01B009017EB0A0918EB050010F1C7
:10C9B000180B009A49465846FEF784F9BDE8F18FF6
:10C9C000F0B583B004000D00002600272068C0F3F6
:10C9D000C5000600382E02D2D6F1380701E0D6F1A4
:10C9E00078070822210000A800F012F83A00DFF8CA
:10C9F000E8172000FFF793FF082200A92000FFF7A7
:10CA00008EFF102214F10801280000F001F8F7BD94
:10CA100070B400230024944214D251F823502554BA
:10CA200051F823502D0A2618757051F823502D0CFB
:10CA30002618B57051F823502D0E2618F5705B1C82
:10CA4000241DE8E770BC704770B4002300249442B2
:10CA500011D2655C6618767855EA06256618B678B0
:10CA600055EA06456618F67855EA066540F82350FB
:10CA70005B1C241DEBE770BC70472DE9F043C1B08F
:10CA800004000D00D4F800906668A768D4F80C8004
:10CA90004022290000A8FFF7D7FF17EA060038EA6E
:10CAA0000601084300990818DFF83017081810EB42
:10CAB00009095FEA796916EB090916EA090037EAFC
:10CAC0000901084301990818DFF81417081810EB3A
:10CAD00008085FEA385819EB080819EA080036EA2E
:10CAE0000801084302990818DFF8F8160818C71952
:10CAF0005FEAF73718EB070718EA070039EA07017A
:10CB0000084303990818DFF8E016081886195FEA49
:10CB1000B626BE1917EA060038EA0601084304994A
:10CB20000818DFF8C816081810EB09095FEA7969D8
:10CB300016EB090916EA090037EA090108430599C5
:10CB40000818DFF8AC16081810EB08085FEA385828
:10CB500019EB080819EA080036EA080108430699A3
:10CB60000818DFF890160818C7195FEAF73718EBAE
:10CB7000070718EA070039EA070108430799081868
:10CB8000DFF87416081886195FEAB626BE1917EA88
:10CB9000060038EA0601084308990818DFF85C1611
:10CBA000081810EB09095FEA796916EB090916EA1A
:10CBB000090037EA0901084309990818DFF8401607
:10CBC000081810EB08085FEA385819EB080819EA4A
:10CBD000080036EA080108430A990818DFF8241605
:10CBE0000818C7195FEAF73718EB070718EA0700B4
:10CBF00039EA070108430B990818DFF80C160818E2
:10CC000086195FEAB626BE1917EA060038EA060159
:10CC100008430C990818DFF8F415081810EB0909F7
:10CC20005FEA796916EB090916EA090037EA090192
:10CC300008430D990818DFF8D815081810EB0808F4
:10CC40005FEA385819EB080819EA080036EA0801C3
:10CC500008430E990818DFF8BC150818C7195FEAD1
:10CC6000F73718EB070718EA070039EA0701084306
:10CC70000F990818DFF8A015081886195FEAB6267C
:10CC8000BE1918EA060037EA080108430199081896
:10CC9000DFF88815081810EB09095FEAF96916EB47
:10CCA000090917EA090036EA070108430699081836
:10CCB000DFF86C15081810EB08085FEAF85819EB54
:10CCC000080816EA080039EA060108430B99081813
:10CCD000DFF850150818C7195FEAB74718EB0707C0
:10CCE00019EA070038EA0901084300990818DFF833
:10CCF0003815081886195FEA3636BE1918EA060094
:10CD000037EA0801084305990818DFF820150818C4
:10CD100010EB09095FEAF96916EB090917EA09003E
:10CD200036EA070108430A990818DFF804150818BD
:10CD300010EB08085FEAF85819EB080816EA080033
:10CD400039EA060108430F990818DFF8E8140818B3
:10CD5000C7195FEAB74718EB070719EA070038EA6F
:10CD60000901084304990818DFF8CC14081886193B
:10CD70005FEA3636BE1918EA060037EA08010843AA
:10CD800009990818DFF8B414081810EB09095FEACC
:10CD9000F96916EB090917EA090036EA07010843A1
:10CDA0000E990818DFF89814081810EB08085FEAC5
:10CDB000F85819EB080816EA080039EA0601084392
:10CDC00003990818DFF87C140818C7195FEAB747F9
:10CDD00018EB070719EA070038EA09010843089920
:10CDE0000818DFF86414081886195FEA3636BE1989
:10CDF00018EA060037EA080108430D990818DFF819
:10CE00004C14081810EB09095FEAF96916EB0909D7
:10CE100017EA090036EA0701084302990818DFF803
:10CE20003014081810EB08085FEAF85819EB0808E6
:10CE300016EA080039EA0601084307990818DFF8DE
:10CE400014140818C7195FEAB74718EB070719EA5F
:10CE5000070038EA090108430C990818DFF8F813AD
:10CE6000081886195FEA3636BE1997EA060098EA6E
:10CE7000000005990818DFF8E413081810EB0909F9
:10CE80005FEA397916EB090996EA090078400899B2
:10CE90000818DFF8CC13081810EB08085FEA785878
:10CEA00019EB080899EA080070400B990818DFF898
:10CEB000B4130818C7195FEA374718EB070798EA51
:10CEC000070099EA00000E990818DFF89C1308186B
:10CED00086195FEA7626BE1997EA060098EA0000EE
:10CEE00001990818DFF88413081810EB09095FEAA4
:10CEF000397916EB090996EA09007840049908186F
:10CF0000DFF86C13081810EB08085FEA785819EB83
:10CF1000080899EA0800704007990818D5490818C8
:10CF2000C7195FEA374718EB070798EA070099EA3D
:10CF300000000A990818D049081886195FEA762671
:10CF4000BE1997EA060098EA00000D990818CB4927
:10CF5000081810EB09095FEA397916EB090996EA16
:10CF60000900784000990818C549081810EB08080E
:10CF70005FEA785819EB080899EA080070400399AD
:10CF80000818C0490818C7195FEA374718EB0707A0
:10CF900098EA070099EA000006990818BA490818A3
:10CFA00086195FEA7626BE1997EA060098EA00001D
:10CFB00009990818B549081810EB09095FEA397989
:10CFC00016EB090996EA090078400C990818B0494F
:10CFD000081810EB08085FEA785819EB080899EA76
:10CFE000080070400F990818AA490818C7195FEA85
:10CFF000374718EB070798EA070099EA00000299FB
:10D000000818A549081886195FEA7626BE1976EA37
:10D010000800784000990818A049081810EB090981
:10D020005FEAB96916EB090979EA070070400799C8
:10D0300008189B49081810EB08085FEAB85819EB64
:10D04000080878EA060090EA09000E990818954940
:10D050000818C7195FEA774718EB070777EA09004E
:10D0600090EA0800059908188F49081886195FEAA0
:10D07000F626BE1976EA080078400C9908188B4904
:10D08000081810EB09095FEAB96916EB090979EA92
:10D0900007007040039908188549081810EB080824
:10D0A0005FEAB85819EB080878EA060090EA090028
:10D0B0000A9908187F490818C7195FEA774718EBDB
:10D0C000070777EA090090EA0800019908187A49E9
:10D0D000081886195FEAF626BE1976EA0800784035
:10D0E000089908187549081810EB09095FEAB96929
:10D0F00016EB090979EA070070400F990818704982
:10D10000081810EB08085FEAB85819EB080878EA25
:10D11000060090EA0900069908186A490818C71914
:10D120005FEA774718EB070777EA090090EA0800FB
:10D130000D9908186449081886195FEAF626BE1981
:10D1400076EA08007840049908186049081810EB3E
:10D1500009095FEAB96916EB090979EA0700704025
:10D160000B9908185A49081810EB08085FEAB858D4
:10D1700019EB080878EA060090EA090002990818F5
:10D1800054490818C7195FEA774718EB070777EA89
:10D19000090090EA0800099908184F4908188619EB
:10D1A0005FEAF626BE19206819EB0000206060686F
:10D1B00030186060A0683818A060E06818EB0000C4
:10D1C000E06041B0BDE8F0830123456789ABCDEF56
:10D1D000FEDCBA98765432108004002078A46AD716
:10D1E00056B7C7E8DB702024EECEBDC1AF0F7CF58B
:10D1F0002AC68747134630A8019546FDD89880690E
:10D20000AFF7448BB15BFFFFBED75C892211906BF7
:10D21000937198FD8E4379A62108B44962251EF6C4
:10D2200040B340C0515A5E26AAC7B6E95D102FD65A
:10D230005314440281E6A1D8C8FBD3E7E6CDE1212F
:10D24000D60737C3870DD5F4ED145A4505E9E3A990
:10D25000F8A3EFFCD9026F678A4C2A8D4239FAFF96
:10D2600081F6718722619D6D0C38E5FD44EABEA40C
:10D27000A9CFDE4B604BBBF670BCBFBEC67E9B2801
:10D28000FA27A1EA8530EFD4051D880439D0D4D916
:10D29000E599DBE6F87CA21F6556ACC4442229F46C
:10D2A00097FF2A43A72394AB39A093FCC3595B652E
:10D2B00092CC0C8F7DF4EFFFD15D84854F7EA86FFB
:10D2C000E0E62CFE144301A3A111084E827E53F721
:10D2D00035F23ABDBBD2D72A91D386EB70B596B062
:10D2E00004000D00160000A8FFF708FB3200210023
:10D2F00000A8FFF714FB290000A8FFF761FB16B098
:10D3000070BD00002248704700B589B02048007801
:10D310008DF818001E4840788DF819001C48807858
:10D320008DF81A001A48C0788DF81B00184800794B
:10D330008DF81C00164840798DF81D00144880793E
:10D340008DF81E001248C0798DF81F001048007A31
:10D350008DF820009DF81F0005909DF82000049096
:10D360009DF81C0003909DF81D0002909DF81E0082
:10D3700001909DF81A0000909DF81B309DF8182030
:10D380009DF819100348F9F7FCFF09B000BD000033
:10D3900028FE000844F900082DE9F04FA1B08046AE
:10D3A000002017461D4602910B900DF1440A6FF0C4
:10D3B00000490AE017F8011B0298C04700280290B4
:10D3C00000F0AB820B98401C0B90387808B90B9892
:10D3D000A5E22528EED10020059006900790089040
:10D3E00009900A9001E040F0010017F8011F202980
:10D3F000F9D023290DD02B2904D02D2906D030298E
:10D400000AD00CE040F0020080B2EEE740F00400E9
:10D41000FAE740F00800F7E740F01000F4E72A29A7
:10D420000ED12968296051F8042B2960002A0D9239
:10D4300004D5514240F004000D9180B27F1C11E0F0
:10D4400000210D9109E00D99494505D001EB8103BB
:10D4500002EB430130390D917F1C3A78A2F1300183
:10D460000A29F0D339782E2903D04FF0FF310C91DF
:10D470001DE017F8011F2A2907D1296829607F1CA0
:10D4800051F8042B29600C9211E000210C9109E065
:10D490000C99494505D001EB810302EB430130397A
:10D4A0000C917F1C3A78A2F130010A29F0D3ADF833
:10D4B00038000FF67840397801F0E2F808B117F833
:10D4C000010B8DF83A009DF83A00682802BF3978C0
:10D4D0006829622005D06C2804BF38786C2803D1F5
:10D4E00071208DF83A007F1C11A8049017F8014BA9
:10D4F000B4F1250029D01C3800F0C280001F02289A
:10D5000040F2BE80133800F0E380093800F0B880A4
:10D51000801E00F04A81401E00F02381401E022838
:10D5200040F2AE80001F00F01C81401F79D0401EE9
:10D5300000F0CE80401E24D0C01E0BD0801E00F014
:10D54000C780C01E00F0C48039E125208DF844005A
:10D5500001203DE12868286050F8046B286003969C
:10D560000C9C002C04D5304600F032FE044606E048
:10D5700022460021304601F08FF800B1841B06944A
:10D5800027E1296829603C2451F8040B2960002117
:10D59000CDE9000111A80390DDE90001049E11B955
:10D5A00008B90C9AB2B10206120FA0EB0212303287
:10D5B000D2B2631E3A2AA8BF2732000940EA01709E
:10D5C00009099A5508BF00281C4603D0039AA319DD
:10D5D0009A42E8D3A0190390C4F13C010C9806913B
:10D5E000814209DA401A08904FF6EF71BDF8380011
:10D5F0000840ADF83800ECE0002840F1EA809DF8E2
:10D60000380000F01400102840F0E3800D98059ACF
:10D61000801A089A801A441A012CC0F2DA80089401
:10D62000D7E09DF83A0062281AD0682806D06A2808
:10D630000CD06C281CD0712808D019E0286828600C
:10D6400050F8041B28600B980880C2E02868286006
:10D6500050F8042B28600B98C117C2E90001B8E00C
:10D660002868286050F8041B28600B980870B0E008
:10D670002868286050F8041B28600B980860A8E010
:10D680002868C01D20F007022A60D2E90001083294
:10D690002A60CDE90001002902D505982D210AE074
:10D6A000BDF83800810702D505982B2103E0C0079B
:10D6B00005D50598202100F80A10401C059011A8F6
:10D6C000059908180390214600A800F0E5F980E0CC
:10D6D0009DF83A006C280DD0712818BF6A2809D12E
:10D6E0002868C01D20F007022A60D2E90001083234
:10D6F0002A6005E02968296051F8040B296000219F
:10D70000CDE900019DF83A00682803D1DDE9000168
:10D7100080B20BE0622803D1DDE90001C0B205E070
:10D72000742818BF7A2804D1DDE900010021CDE971
:10D7300000019DF8380000072ED5DDE90001002921
:10D7400008BF002828D044F02000782824D105986C
:10D75000302100F80A10401C411C059100F80A40D5
:10D760001AE09DF83A00294600F0DCF8CDE9000106
:10D77000002902DA05982D210AE0BDF8380081075A
:10D7800002D505982B2103E0C00705D50598202177
:10D7900000F80A10401C059011A80599081803907C
:10D7A000214600A800F0F5F813E001200590286854
:10D7B000286050F8041B28608DF8441009E02520EB
:10D7C0008DF84400012005901CB18AF80140022028
:10D7D00005900D980599401A0899401A0699401A23
:10D7E0000999401A0799401A0A99441A9DF8380075
:10D7F000400710D420208DF84000002609E00123C6
:10D8000010AA00A9404600F07AFC002840F085806C
:10D81000761CA642F3DB059E0DF1440B0AE01BF8D3
:10D82000011B0298C0470028029076D00B98401C3C
:10D830000B90761E002EF2D130208DF840004FF074
:10D84000000B089E09E0012310AA00A9404600F041
:10D8500056FC002861D10BF1010BB345F3DB069EAA
:10D86000DDF80CB00AE01BF8011B0298C047002845
:10D87000029052D00B98401C0B90761E002EF2D1D5
:10D8800030208DF840004FF0000B099E09E0012385
:10D8900010AA00A9404600F032FC00283DD10BF14F
:10D8A000010BB345F3DB03980699079E01EB000BD0
:10D8B00009E01BF8011B0298C047029068B30B985F
:10D8C000401C0B90761E002EF3D130208DF84000C6
:10D8D0004FF0000B0A9E08E0012310AA00A9404661
:10D8E00000F00DFCC8B90BF1010BB345F4DB9DF85A
:10D8F000380040077FF569AD20208DF840000026F4
:10D9000000E0761CA642BFF660AD012310AA00A974
:10D91000404600F0F4FB0028F3D04FF0FF3021B078
:10D92000BDE8F08F622826D068281DD06A2808D06C
:10D930006C2827D0712804D0742823D07A280CD0E2
:10D9400020E00868C01D20F007000860D0E900232F
:10D95000083008601946104670470A680A6052F895
:10D96000040B0A60002170470A680A6052F8040B31
:10D970000A6000B20BE00A680A6052F8040B0A6001
:10D9800040B204E00A680A6052F8040B0A60C1174A
:10D9900070472DE9FA4E05460A462F696F2A08BFDF
:10D9A000082405D041F02000782814BF0A24102450
:10D9B0003C26D5E90001642A18BF692A81468A46B7
:10D9C00005D1002903DAD9F100096AEB4A0ABAF154
:10D9D000000F08BFB9F1000F0CD1286B50B9082C0B
:10D9E00036D195F83800000732D530203B2687F82D
:10D9F0003B002DE0E31748465146224600F078FEF2
:10DA0000A4FB0023A9EB02023032D2B2A6F1010B33
:10DA10003A2A5E4603DB9DF80030513B9A18814656
:10DA20005FEA010A0BF8072008BFB9F1000F03D025
:10DA3000E868F1198842DDD3082C09D195F838003F
:10DA4000000705D5F05D302802D0761E3020F05555
:10DA5000C6F13C00A861F119E960296B884208DA37
:10DA6000081A28624FF6EF71288F08402887BDE812
:10DA7000F38E00290ED595F8381001F01401102905
:10DA800008D1696B6A69891A2A6A891A0E1A012EE5
:10DA9000A8BF2E62BDE8F38E2DE9F24F04468EB08A
:10DAA000D4E90001CDE9020104AF9DF8380040F04F
:10DAB000200BBBF1610F0AD0206B002848BF062065
:10DAC00004D408BFBBF1670F01D101202063616856
:10DAD000C1F30A5040F2FF7290421CD1080304BF08
:10DAE0002068002809D10320A0619DF83800613822
:10DAF0001A2836D30FF2486108E00320A0619DF890
:10DB0000380061381A2829D30FF22C61E06803220B
:10DB1000FDF7D8F8BEE1012816DA204600F05FFED6
:10DB2000012811DB00250020BBF1610F20D1E16845
:10DB3000302201F8012B4A1CE2609DF83820612A4E
:10DB40000CBF782258220FE0626840F2FE3161F388
:10DB50001E52451A62604FF0FF30E5E70FF2D451D4
:10DB6000D4E70FF2D851D1E70A706169891C61616D
:10DB700010B90026002584E1BBF1610F40F09780C9
:10DB8000206BD4E900AB00284CBF2126461CDDE900
:10DB900002010022002300F043FE36B23ABF8BF0B0
:10DBA0000040CDE902A0CDE902AB06F101082D1F2E
:10DBB0008DF810200DF1110700E0C71DB8F1010F1D
:10DBC00033DBDDE902010022002300F041FE2CD20C
:10DBD0001C2102A800F054FEDDE9020100F0D8FE8D
:10DBE000A8F10708B8F1010F814609DB00F0FCFE3F
:10DBF00002460B46DDE9020100F00EFFCDE902010D
:10DC0000F81D072105E009F00F0200F8012D4FEA89
:10DC10002919B9F1010F01DB491EF4D5491E5CBF7A
:10DC2000002200F8012DF9D5C7E70DF11100391ACE
:10DC3000B142B8BF0E4636B230000DF111072FD4F5
:10DC4000884206DA04A9411849780829A8BF0F219B
:10DC500000DA002104AA821800E0761E12F80139C9
:10DC6000401E8B42F9D00F2904D104A941184A78EB
:10DC7000521C4A70002802D504AF761C2D1D36B206
:10DC8000701E0DD4C1190A783032D2B23A2A03DBA1
:10DC90009DF838303A3B9A18401E01F80129F2D518
:10DCA000206B002840F1ED80701E2063E9E0DDE983
:10DCB00002010022002300F0B3FD3CBF81F00041CF
:10DCC000CDE902012DB247F2975068434B49DFF886
:10DCD000309190FBF1F52DB2C5F1070ABAF1010FB1
:10DCE00090461CDBDDE902675FEACA7007D5424651
:10DCF0004B463046394600F04FFF06460F46404639
:10DD0000494642464B464FEA6A0A00F045FFBAF1DF
:10DD1000000F80468946E7D1CDE9026724E0CAF1C9
:10DD2000000A0026374F14E05FEACA7007D5424662
:10DD30004B463046394600F02FFF06460F46404618
:10DD4000494642464B4600F027FF4FEA6A0A8046A2
:10DD50008946BAF1000FE7D1DDE9020132463B46C0
:10DD600000F0ECFFCDE90201BBF1660F216BDFF89B
:10DD700098900CBF05F10A0006204618142EA8BF83
:10DD8000132630208DF810000DF11107012E3DDB18
:10DD9000DDE9020100F012FE07F1080104220A2366
:10DDA000B0FBF3F303EB8307A0EB4700303001F83F
:10DDB000010C0A20B3FBF0F000EB8007A3EB470354
:10DDC0003033521E01F8023DE9D1083E012E01F127
:10DDD0000807DBDBDDE9020100F0F0FD00F00EFEDC
:10DDE00002460B46DDE9020100F016FE00224B461A
:10DDF00000F0D2FECDE90201CAE700BFA086010013
:10DE0000000024400000F03F84D797410DF111003D
:10DE1000381A0DF1110702E0401E6D1E7F1C397883
:10DE20003029F9D0BBF1660F02D12DB2691C04E094
:10DE3000BBF1650F0CBF01210021226B8E1836B299
:10DE4000B042B8BF064636B231001AD4814204DA75
:10DE5000C85D3528A8BF392000DA3020CA19521E03
:10DE600000E0761E12F80139491E8342F9D03928A4
:10DE700002D1C85D401CC855002902D57F1E761C02
:10DE80006D1C2DB29DF83810009533B23A462046ED
:10DE900000F003F80FB0BDE8F08F2DE9F043054620
:10DEA0001E46D5F83080012E85B08946174602DA25
:10DEB00001260FF2902749F02000BDF93040662876
:10DEC00008BF641C17D0672840F0828014F1040F4B
:10DED000C0F28480444580F2818095F83800641C4B
:10DEE000000702D44645B8BFB04624B2B8EB0408D8
:10DEF00048BF4FF0000824B2E868A969012C25DA70
:10DF00004A1C30230B54B8F1010F03DA95F838108E
:10DF1000090702D52E211154521C18EB040FB8BF6B
:10DF2000C8F1000424B2A0446142B045AA6169620C
:10DF3000B8BF4646AB6936B2EE613246394618186C
:10DF4000FCF7C0FEA8EB0600A862C1E00818A642D4
:10DF500018DA32463946FCF7B5FEA9697118A01BDC
:10DF6000B8F1010FA961686203DA95F8380000077B
:10DF700005D5EA682E208854E869401CE861C5F898
:10DF80002880A5E022463946FCF79CFEA8692018A7
:10DF9000361BB8F1010F03DA95F83810090703D5DD
:10DFA000EA682E218154401CA86136B2B045B8BF42
:10DFB0004646E868AB6936B23246E1191818FCF7F4
:10DFC00081FEA8693018A861A8EB060068627FE0AE
:10DFD000B9F1610F16D14FF0700918E0464504DA27
:10DFE00095F83810090758BFB046B8F1010848BF86
:10DFF0004FF00008B9F1670F14BF4FF045094FF01B
:10E00000650904E0B9F1410F08BF4FF05009A96953
:10E01000E86817F8013B0B544A1CB8F1010F05DA08
:10E0200095F83810090758BFAA6117D52E21115449
:10E03000531CB8F1010FAB6110DB761E36B2B04550
:10E04000B8BF464636B2324639461818FCF73AFE93
:10E05000A8693018A861A8EB06006862E868A96999
:10E060000918200081F8009003D42B2048708F1CE1
:10E0700003E02D224A708F1C644200260DF108082F
:10E0800008E00A2200A800F084FF019808F8010BBC
:10E09000761C009C21B20129F3DA022E06DA49F03F
:10E0A0002000652804BF302007F8010B4EB930204E
:10E0B00007F8010B07E0761E02A8305C303007F845
:10E0C000010B012EF7DAE868A9690818381AE86127
:10E0D00095F8380000F0140010280DD16869A9697E
:10E0E0000818696A0818E9690818A96A0818696BA4
:10E0F0008842BCBF081A286205B0BDE8F083F8B5B5
:10E1000004460D4616461F46002004E0E86A401CFF
:10E11000E8627F1E002047B116F8011BA868A047DF
:10E120000028A860F2D14FF0FF30F2BD686A6C742D
:10E130007A4C00006E616E004E414E00696E6600C2
:10E14000494E460030000000EFF30980BFF36F8FA7
:10E150001D4B1A6820E9F00F106008B54FF0100051
:10E1600080F31188BFF34F8FBFF36F8FF9F781FEF4
:10E170004FF0000080F31188BDE808401968086876
:10E18000B0E8F00F80F30988BFF36F8F70470E4B34
:10E1900019680868B0E8F00F80F30988BFF36F8F43
:10E1A0004FF0000080F311884EF00D0E70470748C5
:10E1B0000068006880F3088862B661B6BFF34F8FCD
:10E1C000BFF36F8F00DF0000E886002008ED00E05D
:10E1D00000F10103810704D010F8011B89B1810708
:10E1E000FAD10268B2F10131914311F0803F04BFCE
:10E1F00050F8042FF6E710F8011B11B110F8011BBD
:10E20000FBE7C01A7047002300F0CABE002200F0EE
:10E210000BBF70B504001A250026E4B2002C01D112
:10E220000124FFE7E4B2EDB2AC4201D32C00FFE7DA
:10E23000E4B29C2000FB04F006007D20FBF7B1FF58
:10E24000002801D0FBF7D5FF45F2555000F00CF83F
:10E25000062000F00DF8300080B200F00DF800F05C
:10E260000FF800F012F870BD80B20A4908607047DC
:10E27000C0B209490860704780B208490860704719
:10E280004AF6AA200349086070474CF6CC40014981
:10E290000860704700300040043000400830004003
:10E2A00080B50120FBF779FF01BD80B50A495FF019
:10E2B0000060FCF71CFA05208DF8000000208DF8A6
:10E2C000010000208DF8020001208DF8030000A855
:10E2D000FCF7D7F901BD00000050000880B5082008
:10E2E000FBF78EFF00280AD00820FBF797FF3120AC
:10E2F000FBF757FF002802D00120FBF7A1FE1020FA
:10E30000FBF77EFF00280AD01020FBF787FF39209B
:10E31000FBF747FF002802D00220FBF796FE01BD65
:10E3200080B57648006850F0010074490860744870
:10E330000068744908407249086070480068724972
:10E3400008406E4908606D48006830F480206B49D1
:10E3500008606B48006830F4FE00694908605FF4AB
:10E360001F006A49086000F054F85FF000606849D7
:10E37000086001BD10B4002000210022604B1B6822
:10E3800013F00C0318000300002B04D0042B06D05C
:10E39000082B08D02BE05F4B5F4C23602AE05F4BDB
:10E3A0005D4C236026E0564B1B6813F47013190074
:10E3B000534B1B6813F480331A00890C891C002A04
:10E3C00005D1574B03FB01F3534C23600EE04C4B3C
:10E3D0001B689B0305D54F4B03FB01F34E4C236099
:10E3E00004E04E4B03FB01F34B4C236002E0494B2E
:10E3F000494C2360424B1B684A4CC3F303131B5D1B
:10E400001800454B1B681C00C440434B1C6010BCEB
:10E41000704780B500F001F801BD82B00020019086
:10E42000002000903548006850F48030334908607F
:10E430003248006810F4003000900198401C0190B0
:10E440000098002803D10198B0F5A06FF0D12B48B7
:10E450000068800302D50120009001E000200090B8
:10E460000098012847D13048006850F010002E492C
:10E4700008602D480068800880002B4908602A4801
:10E48000006850F00200284908601D4800681C49D7
:10E4900008601B4800681A4908601948006850F471
:10E4A0008060174908601648006830F47C101449F1
:10E4B00008601348006850F41020114908600F48A4
:10E4C000006850F080700D4908600C4800688001B9
:10E4D000FBD50B480068800880000949086008489F
:10E4E000006850F00200064908600548006810F016
:10E4F0000C000828F9D102B070470000001002405B
:10E50000041002400000FFF8FFFFF6FE0810024072
:10E5100008ED00E000127A00480500200024F40015
:10E5200000093D00D004002000200240DFF808016F
:10E53000DFF808110860DFF80801DFF80011086053
:10E540007047DFF80001006850F08000DFF8F41039
:10E550000860704738B5040004255FF4302000F0EF
:10E5600077F80500EDB2042D20D1DFF8D80000685F
:10E5700050F00200DFF8CC100860DFF8CC00046037
:10E58000DFF8C000006850F04000DFF8B810086005
:10E590005FF4302000F05CF80500DFF8A8000068A8
:10E5A00041F6FD710840DFF89C1008602800C0B2F9
:10E5B00032BD70B504000D0004264FF4005000F089
:10E5C00047F80600F6B2042E16D1DFF8780000688E
:10E5D00050F00100DFF86C10086025804FF4005007
:10E5E00000F036F80600DFF85C00006841F6FE71C6
:10E5F0000840DFF8501008603000C0B270BD134909
:10E6000008607047042011490968C90702D5012133
:10E6100008000FE00D490968490702D502210800EA
:10E6200008E00A490968C90602D50321080001E08B
:10E6300004210800C0B2704723016745042002404E
:10E64000AB89EFCD10200240142002400C20024084
:10E6500038B504000425FFF7D5FF0500EDB2012D04
:10E6600006D1002C04D0FFF7CDFF0500641EF5E7AE
:10E67000002C01D1052005002800C0B232BD704732
:10E680000278C9B28A421AB11CBF10F8012FF9E70B
:10E6900018BF002070470000C9B2830706D0521E81
:10E6A00022D310F8013B9942F7D11FE0083A13D367
:10E6B00002F1040241EA012141EA014150F8043B20
:10E6C000121F21BF4B40A3F1013C2CEA030C1CF0AC
:10E6D000803FF3D0C9B2001F083210F8013B521E30
:10E6E00028BF91EA030FF8D818BF0120401E7047D9
:10E6F0001B4213D1094236D12AB18446B0FBF2F055
:10E7000002FB10C2704700F0A9BCFCD3002200231A
:10E7100070470B000200002100207047904271EB0F
:10E72000030CF6D370B5B1FA81F4B3FA83F52C1B60
:10E73000A340C4F1200532FA05F63343A2405FF04E
:10E740000046E64002E05B085FEA3202841A71EBA1
:10E75000030524BF204629467641F4D302000B006E
:10E760003000002170BD012ACFD970B5140C20D023
:10E77000B1FA81F4B2FA82F5C4F120046419B4F15B
:10E780002006D6D3B2405FF00044F440002502E0FA
:10E7900052085FEA3303C61A71EB020E24BF3046FB
:10E7A000714664416D41F3D302000B002000290043
:10E7B00070BD0C46B1FBF2F102FB11452D0445EA98
:10E7C0001045B5FBF2F402FB145580B240EA054552
:10E7D000B5FBF2F002FB105240EA044070BD30B4C9
:10E7E000436803F0004201211B031B0B436004BF7D
:10E7F0000368002B08D10DE00368DD0F45EA4404EF
:10E8000044605B000360491E4468E302F4D52303BF
:10E810001B0B436043681A434260084630BC704794
:10E820004FF4001C1CEB410F94BF1CEB430F09E09D
:10E8300041EA030C50EA4C0C52EA0C0C03D2994208
:10E8400008BF9042704714BF8B428242704700005D
:10E850004FF4001C1CEB410F94BF1CEB430F09E06D
:10E8600041EA030C50EA4C0C52EA0C0C03D28B42E6
:10E8700008BF8242704714BF99429042704700001F
:10E8800070B504460D466068C0F30A5040F2FF714F
:10E89000884207D16068000304BF2068002817D0B1
:10E8A000022070BD20B92046FFF799FF012868DAE1
:10E8B000012D0FDB40F2FF71091A8D420AD3606807
:10E8C000002847BF0020304900203049C4E900013A
:10E8D000012070BD4142A942616806DA6FF31E5102
:10E8E000401941EA0050606042E0401E63684519EB
:10E8F000012205F1350062F31F53352801F0004174
:10E90000636003D361600020206070BD002215F1B8
:10E910001F0F04DA226823600020203560606842FF
:10E9200014D0521E25689241C0F12003D2439D406D
:10E9300045EAD272256825FA00F6656805FA03F300
:10E9400033432360636823FA00F565606068084319
:10E95000B2F1004F606003D80DD12078C0070AD50E
:10E960002068401C2060206828B96068401C6060F6
:10E970004FF0FF3070BD6068884204BF20680028F7
:10E98000F6D1002070BD00BF0000F0FF0000F07F56
:10E99000F446400D40EAC120490006D200F014F8C8
:10E9A000004248BF6FF00040604700F00DF84FF0A4
:10E9B000004188428CBF084640426047400D40EA13
:10E9C000C120490080F00D8040F00040490DA1F5C4
:10E9D0008061491C05D4D1F11F0154BFC840C01744
:10E9E00070474FF000007047010040F10980F44685
:10E9F000404200F005F851F000416047010000BFBF
:10EA000009D0B0FA80F18840C91CC1F584610905BC
:10EA100001EBD02140057047F0B44FF0004591EA7A
:10EA2000030F44BF6B4000F01BBB00BF841A71EBA7
:10EA3000030604D26E40001BB141121973414FF41A
:10EA4000001C1CEB410F34BF7CEB430684E00C0D33
:10EA5000A4EB1356362E7DDC012E43DC45EAC3239E
:10EA600043EA525312BFD20292025B08240545EAE0
:10EA7000C12141EA5051D2EBC020994125D407D1A0
:10EA8000B0FA80F610FA06F164D00020203608E0D3
:10EA9000B1FA81F6B140C6F1200220FA02F2114328
:10EAA000B0404FEAF474B4EB465434F001064FEA38
:10EAB00074040AD8D6F50016760D04F00044F04030
:10EAC00061FA06F25040F1404840C00A40EA415025
:10EAD00021F0004128BF5FEA500550F1000044EBEF
:10EAE000D12137E045EAC323DB0A45EAC121C90A3F
:10EAF000B6F120050EDD42EA0242120CC5F12006F5
:10EB000003FA06F6EB4042EA06056D42984161F1D0
:10EB100000010DE062FA06F5F240554063FA06FC8A
:10EB200082EA0C02F3405A406D42904161EB0301CE
:10EB300011F4801F05D1641E620502D06D004041B2
:10EB4000494121F48011430875F1004350F1000060
:10EB500041EB0451F0BC70471CEB410F15D223F080
:10EB6000004352EA43060BD04FEA4C0CBCEB410F7A
:10EB700004D80C0D661E342EB7DDEBE7801A9941E0
:10EB800050EA410608BF0021E4E708BF1CEB430F31
:10EB900028BF6FF00001DDE7B0B581EA030C0CF08F
:10EBA000004C40F2FF7515EA11541DBF15EA1357CA
:10EBB000AC42AF4239E0E41923EA455343F48013F1
:10EBC000C90241F0004141EA505EC7021100A7FBB3
:10EBD000020200284FF00000EEFB01204FF0000180
:10EBE000E3FB072118BF42F0010240180021494110
:10EBF000E3FB0E01A4F580640F0302D252004041F2
:10EC0000494154F101046CDD470872F1004250F1B2
:10EC1000000051EB0451A1F580115CBF41EA0C01E9
:10EC2000B0BD4CEA05510020B0BD05EA1357AC4217
:10EC300014BFAF4241E050EA410E1CBF52EA430EFE
:10EC400002E061460020B0BD24423C441BD15FEA93
:10EC5000070EF6D0090302BF01460020AEF1140EE4
:10EC6000B1FA81F7AEEB070401FA07FE0C37C7F1E2
:10EC7000200100FA07F7C8404EEA000E23EA455388
:10EC800043F48013A2E733F00043B3FA83F704BFE1
:10EC9000B2FA82FE77440B3FE41BB7F1200E2FBF80
:10ECA00002FA0EF3BB40C7F1200E22FA0EFE38BF67
:10ECB00043EA0E03BA40641C82E750EA410E14BFD7
:10ECC00052EA430E6FF000014FF4001717EB430FA9
:10ECD0008ABF194617EB410FB5E74CEA05510020F2
:10ECE000B0BDD4F10104B4F120070FDAC4F120075C
:10ECF000520828BF42F0010210FA07F501FA07F79F
:10ED0000E1BF2A43E0403843E1400FE0352C98DC76
:10ED1000C7F1200452EA400220FA07F218BF42F07D
:10ED2000010231FA07F0A1400A43002172F10042CA
:10ED300050F1000051EB0C01B0BD00002DE9F04195
:10ED400040F2FF7581EA030C0CF0004C15EA1154F7
:10ED50001DBF15EA1357AC42AF42E9E0BC41C1F315
:10ED60001301C3F31303801A994143F4801304D2AF
:10ED7000641E4000494180185941C90241EA50517E
:10ED8000B1FBF3F603FB1611A2FB0675D7EBC0200F
:10ED9000A94102D2761E80185941C90241EA505158
:10EDA000B1FBF3FE03FB1E11A2FB0E75D7EBC020D7
:10EDB000A94103D2AEF1010E80185941890241EAFE
:10EDC0009051760546EA8E2EB1FBF3F603FB161141
:10EDD000A2FB0675D7EB8020A94102D2761E8018CF
:10EDE0005941C90241EA50514EEA060EB1FBF3F611
:10EDF00003FB1611A2FB0675D7EBC020A94102D276
:10EE0000761E80185941C90241EA5051B1FBF3F70F
:10EE100003FB1711A2FB0735D3EBC020A94167F113
:10EE200000070CBF004247F0010766F3D5274FEA01
:10EE30001E31B80814F5806414DDBD0775F1004279
:10EE400050EB0E5051EB045111F5801F5CBF41EAAD
:10EE50000C01BDE8F0814CF07F6141F0E041002001
:10EE6000BDE8F081BD076D0840EA0E5041F4801105
:10EE7000D4F10104B4F120060ADAC4F1200602003C
:10EE8000E04001FA06F3E1401843B24015430EE0BA
:10EE9000342C14DCC6F1200445EA40056D0820FA44
:10EEA00006F2154321FA06F0A1400D43002175F149
:10EEB000004250F1000051EB0C01BDE8F081002050
:10EEC0005FEA0C01BDE8F081CFB992185B41B3FA5B
:10EED00083F704BFB2FA82F6BF190B3FB7F12006E1
:10EEE0002FBF02FA06F3BB40C7F1200622FA06F64E
:10EEF00038BF3343BA401CB1E419641E2FE77F4288
:10EF000031F00041B1FA81F404BFB0FA80F6A419DF
:10EF10000B3CB4F120062FBF00FA06F1A140C4F16A
:10EF2000200620FA06F638BF3143A0403C1B16E706
:10EF3000AC421ABF05EA1357AF4214E050EA41064B
:10EF40001CBF52EA4306BFE750EA4107304661461C
:10EF50001CBF41EA0551BDE8F08152EA430C08BFED
:10EF6000C143BDE8F08100204FF4001616EB410FBD
:10EF700098BF16EB430F08BF16EB410F24BFC143E8
:10EF800005E016EB430F0CBF61464CEA0551BDE8A6
:10EF9000F08191FBF2F303FB1211C0E900317047DD
:10EFA0002DE9F04182B080460E001D4608BF00AE3C
:10EFB000474600E07F1C3878A0F109010529F9D304
:10EFC0002028F7D02D2816BF2B2817F8014B2B240B
:10EFD0003146384600F0AEF831688F4208BFC6F8B7
:10EFE00000803168884514D120B92D2C16D1B0F19C
:10EFF000004F15D900F06AF9222101600DB10120FE
:10F0000028602D2C14BF6FF000404FF00040BDE889
:10F01000F6812B2CE9D1B0F1004FEBD2BDE8F6819F
:10F020004042BDE8F681000000B500BF13009646DF
:10F030009446103928BFA0E80C50FAD85FEA417C0A
:10F0400028BF0CC048BF40F8042BC90728BF20F8D0
:10F05000022B48BF00F8012B00BD000070470000E4
:10F06000841A71EB030603D2001BB14112197341DC
:10F070004FF4001C1CEB410F34BF7CEB430443E016
:10F080000C0DA4EB1356352E50DC45EAC323DB0AE6
:10F0900045EAC121C912B6F120050DDD63FA05F676
:10F0A000EB4086EA0305124218BF45F00105C0187F
:10F0B00051F100010CD213E062FA06F5F24055401E
:10F0C000F3415A40B340F3405A408018594107D3A6
:10F0D00049085FEA30005FEA350528BF45F00105C1
:10F0E00001F58011420875F1004250F1000041EB3A
:10F0F0000451F0BC4FF4001C1CEB410F38BF7047AB
:10F100000020090D090570471CEB410F10D252EA8F
:10F1100043060BD0BCEB410F05D80C0DAB43661E6C
:10F12000342EB5DD02E0AB4380185941F0BC704786
:10F13000F0BC70472DE9F04F85B004461E000D4627
:10F1400090461CBF00203060A14601E009F1010992
:10F1500099F80000A0F109010529F7D32028F5D07E
:10F160002D2816BF2B2819F8017B2B27B8F1000F8B
:10F1700057D4B8F1010F54D0B8F1250F51DAB8F1D6
:10F18000010F0DDBB8F1100F04BF99F80000302813
:10F1900002BF99F8010040F02000782814D10EE059
:10F1A00099F80000302818BF4FF00A080CD199F8E0
:10F1B000010040F02000782804D14FF0100809F138
:10F1C000020901E04FF00808CDF8109001E009F1C4
:10F1D000010999F800003028F9D00FF2A00B4FF088
:10F1E000000ACDF80C908DF808B00AE09DF80810E0
:10F1F000CDF804A0401AC0B2009008FB0A0A09F139
:10F20000010999F80010A1F141001A2838BF2031F6
:10F2100042465846FFF740FA0028E7D1049848458F
:10F2200003D105B12C60002025E00FF2780103988E
:10F2300018F80110A9EB0000401A14D4012808DACC
:10F240000098BAEB000004D30199B0FBF8F08842B3
:10F2500009D000F03BF8222101600EB1012030609E
:10F260004FF0FF3A03E02D2F08BFCAF1000A0DB19D
:10F27000C5F80090504605B0BDE8F08F303132330C
:10F280003435363738396162636465666768696A40
:10F290006B6C6D6E6F707172737475767778797A46
:10F2A0000000000000002115110E0D0C0B0B0A0AC6
:10F2B00009090909090808080808080807070707CD
:10F2C0000707070707070707070000000148FFF7C0
:10F2D000D6B90000580500200000891112239B3286
:10F2E0002446AD573665BF74488CC19D5AAFD3BE16
:10F2F0006CCAE5DB7EE9F7F88110080193331A2226
:10F30000A5562C47B7753E64C99C408DDBBF52AEF5
:10F31000EDDA64CBFFF976E802218B301002991305
:10F320002667AF763444BD554AADC3BC588ED19FD5
:10F330006EEBE7FA7CC8F5D983310A2091121803E5
:10F34000A7772E66B5543C45CBBD42ACD99E508FB5
:10F35000EFFB66EAFDD874C904428D5316619F70B5
:10F360002004A9153227BB364CCEC5DF5EEDD7FC95
:10F370006888E1997AABF3BA85520C4397711E60A5
:10F38000A1142805B3373A26CDDE44CFDFFD56EC75
:10F39000E9986089FBBB72AA06638F7214409D5185
:10F3A0002225AB343006B9174EEFC7FE5CCCD5DD55
:10F3B0006AA9E3B8788AF19B87730E6295501C4165
:10F3C000A3352A24B1163807CFFF46EEDDDC54CD35
:10F3D000EBB962A8F99A708B088481951AA793B645
:10F3E0002CC2A5D33EE1B7F04008C919522BDB3A35
:10F3F000644EED5F766DFF7C899400859BB712A605
:10F40000ADD224C3BFF136E0C1184809D33B5A2A14
:10F41000E55E6C4FF77D7E6C0AA583B418869197E4
:10F420002EE3A7F23CC0B5D14229CB38500AD91BF4
:10F43000666FEF7E744CFD5D8BB502A499961087C4
:10F44000AFF326E2BDD034C1C3394A28D11A580BD4
:10F45000E77F6E6EF55C7C4D0CC685D71EE597F494
:10F460002880A1913AA3B3B2444ACD5B5669DF78B4
:10F47000600CE91D722FFB3E8DD604C79FF516E484
:10F48000A9902081BBB332A2C55A4C4BD7795E6894
:10F49000E11C680DF33F7A2E0EE787F61CC495D564
:10F4A0002AA1A3B03882B193466BCF7A5448DD5974
:10F4B000622DEB3C700EF91F8FF706E69DD414C544
:10F4C000ABB122A0B9923083C77B4E6AD5585C4954
:10F4D000E33D6A2CF11E780F816807E0026811682D
:10F4E000536889185B18C36008320260C268914291
:10F4F000F4D04A1C82600878704738B504460D463F
:10F50000A068E168884212D120686168884208BF1B
:10F5100000F0C3F82068227C016802B14944A16070
:10F5200042685218E260083091422060ECD0A06836
:10F53000401CA06000F8015D31BD2DE9F0418AB0AA
:10F5400000F1080105910268520801EBC201069121
:10F550000021079108910168490800EBC1010831B9
:10F560000091017901F001018DF8101040680099B7
:10F57000400801EBC000019000200290039084E05D
:10F5800005A8FFF7A9FF044614F0030603D105A858
:10F59000FFF7A2FFC61C25090F2D1BD105A8FFF7F9
:10F5A0009BFF00F10F0515E0059801680818059903
:10F5B0000790496808180890059808300590079842
:10F5C00008998842F0D0401C079010F8011D00A84F
:10F5D000FFF793FF761EF2D1002D51D005A8FFF75B
:10F5E0007BFF0646A00800F00300032804BF05A81F
:10F5F000FFF772FFDDF800800299039F06EB002001
:10F6000008E0A8F10808A8F10801801A0A6849680A
:10F610008F18394658F8082C8A1A8242F1D30C1AEE
:10F62000AE1C2DD0BC4206D158F8044B58F8040B40
:10F630000719BC42F8D00298039914F8015B88427C
:10F6400017D100980199884208BF00F026F8009869
:10F6500000689DF81010029009B14844029000998A
:10F6600002984968009A091808328842039100926A
:10F67000E7D00298401C0290761E00F8015DD1D1BF
:10F680000298039988427FF47BAF019800998142E8
:10F690007FF476AF0AB0BDE8F081012000F000B839
:10F6A00080B5C046C046024A11001820ABBEFBE739
:10F6B0002600020034FE000873BF000800000000AE
:10F6C00040FE0008F9BF0008000000004CFE0008E2
:10F6D00029C0000800000000DCFE0008EDC00008A2
:10F6E0000000000058FE00080DC1000800000000E6
:10F6F00064FE0008F9A500080000000070FE000884
:10F7000081A50008000000007CFE00084FA500084D
:10F7100000000000E4FE000835C100080000000001
:10F72000ECFE00084DC1000800000000F4FE0008D7
:10F7300067C100080000000034FF000809D300087A
:10F7400000000000FCFE000809970008000000000F
:10F7500053544D33325F466C6173685772697465F8
:10F76000204572722070726F6772616D41646472BD
:10F77000203D20253038782073697A65203D20258A
:10F7800064206F6666736574203D20256420737461
:10F7900061747573203D2025640D0A00453A5C674D
:10F7A000697450726F6A6563745C66726565525401
:10F7B0004F535F4D6F64656C5F70726F6A65637401
:10F7C0005C536F757263655C706F727461626C65B7
:10F7D0005C4D656D4D616E675C686561705F342E70
:10F7E00063000000453A5C67697450726F6A656334
:10F7F000745C6672656552544F535F4D6F64656CFF
:10F800005F70726F6A6563745C536F757263655C79
:10F81000706F727461626C655C4941525C41524D1B
:10F820005F434D335C706F72742E630019E050F8C3
:10F83000041BCB0744BFA9F101035918121F002371
:10F84000042A41F8043BF9D25FEA827C0B4604D5D6
:10F850004FF0000CA1F800C09B1CD10744BF002151
:10F86000197050F8042B002AE1D1704753544D33DE
:10F87000325F466C6173685061676545726173659C
:10F8800020457272207061676541646472203D207A
:10F890002530387820737461747573203D20256499
:10F8A0000D0A0000453A5C67697450726F6A6563BF
:10F8B000745C6672656552544F535F4D6F64656C3E
:10F8C0005F70726F6A6563745C536F757263655CB9
:10F8D00074696D6572732E6300000000453A5C67C1
:10F8E000697450726F6A6563745C667265655254C0
:10F8F0004F535F4D6F64656C5F70726F6A656374C0
:10F900005C536F757263655C71756575652E630018
:10F91000453A5C67697450726F6A6563745C6672BD
:10F92000656552544F535F4D6F64656C5F70726FC5
:10F930006A6563745C536F757263655C7461736B45
:10F94000732E630041504C2056657273696F6E3D93
:10F9500025632563256325632D25303278253032D4
:10F9600078253032782D56253032782E2530327871
:10F970000D0A000010B5074979441831064C7C4443
:10F98000163404E00A68081D511888470146A14250
:10F99000F8D110BD740000009C0000006D65746516
:10F9A00072206661696C6564206D6F726520746891
:10F9B000616E206D6F73742074696D65730D0A003C
:10F9C00077616974206D62757320736C6176652050
:10F9D00066696E6973682074696D656F75740D0A68
:10F9E0000000000077616974206D627573206D619D
:10F9F000737465722066696E6973682074696D65D9
:10FA00006F75740D0A00000025FEFFFF10820000D4
:10FA1000640500200000000023FBFFFF020000003F
:10FA20000200000034060000550200000000002023
:10FA30006405000063726561746520706F727420E4
:10FA40007853656D6170686F7265206661696C6579
:10FA5000640D0A007570646174652066696C6520C8
:10FA6000696E6469636174696F6E206572720D0AF4
:10FA7000000000000D0A636F6D6D616E64206C659F
:10FA80006E677468206572726F72210D0A00000043
:10FA9000696E70757420686176656E277420737462
:10FAA0006172742061742030780D0A00736C617685
:10FAB0006520636F756E7420657863656564206D7D
:10FAC00061780D0A0000000063616E206E6F742083
:10FAD0006C6F636174696F6E2061206275660D0AD8
:10FAE000000000007265616420666C617368206DBF
:10FAF0006574657220737563636573733A00000003
:10FB00006D62757320736C6176652061636B207420
:10FB10006F2073746174696F6E0D0A007772697477
:10FB200065207061636B657420256420696E2066B2
:10FB30006C6173680D0A0000746F74616C207570DD
:10FB4000647465206279746573203D2025640D0A14
:10FB5000000000007570646174655F746F74616C9F
:10FB60005061636B657473203D2025640D0A0000AD
:10FB700000F00BF8002801D0FFF7FCFE0020C04683
:10FB8000C046FCF7BCFC00F002F80120704700F012
:10FB900001B8000007463846FFF782FDFBE700008A
:10FBA0006E6F6465206973206E6F7420696E206CBF
:10FBB0006973740D0A0000006E6F646520616C72D9
:10FBC000656164792065786973740D0A000000002E
:10FBD00064656C65746520616E206F6C64206E6F67
:10FBE00064650D0A00000000726570656174206133
:10FBF000636B20746F2073746174696F6E3A0000D8
:10FC0000616C6C207061636B6574207265636569FB
:10FC10007665640D0A000000434D443A20B2BBD61D
:10FC2000A7B3D6C3FCC1EE0D0A0000007772697459
:10FC3000652061646472206572720D0A0000000024
:10FC40004D42555320706F77657220686967680D63
:10FC50000A0000004D42555320706F776572206C8A
:10FC60006F770D0A0000000061636B20746F2063E2
:10FC7000616C6C20616464723A0000004D55542040
:10FC8000504F5254205458206E6F6E650D0A00007C
:10FC900075617274207377697463682074696D6527
:10FCA00072000000706C632061636B20746F2073BE
:10FCB000746174696F6E3A0072656164206D657479
:10FCC000657220737563636573733A00726561646E
:10FCD000206D65746572206661696C65643A000028
:10FCE0007468652073616D65207061636B65740D68
:10FCF0000A0000007570646174652066696C652097
:10FD00006572720D0A00000061646472206C656E99
:10FD1000206572720D0A00006C6F63616C20616473
:10FD200064722030780000005461736B2072782078
:10FD30007072696E746600007472616E73706172C5
:10FD4000656E7420303020006C69737420697320F4
:10FD500066756C6C0D0A00006E6F20736C617665C1
:10FD6000206E6F64650D0A006C69737420656D7098
:10FD700074790D0A000000006F70656E207377695A
:10FD80007463680D0A000000504C432053494D55E0
:10FD90004C2052583A000000636C6F7365207377F3
:10FDA000697463680D0A00004D425553206D6173FC
:10FDB0007465722054583A004D425553206D61735A
:10FDC0007465722052583A004D42555320736C614D
:10FDD0007665205258203A0074782074696D656FFA
:10FDE00075740D0A000000004D42555320736C617C
:10FDF00076652054583A0000F00200205403002099
:10FE00001C040020B80300207570646174652073C1
:10FE1000746172740D0A0000014880470148004770
:10FE200021E30008D1FE0008654C67611304170147
:10FE300001000000777269746561646472000000FB
:10FE400072656164616464720000000073696D75BD
:10FE50006C706C6300000000616464666C617368C0
:10FE6000000000007363616E6C6973740000000031
:10FE70007363616E666C617368000000636C726628
:10FE80006C617368000000005461736B20707269CC
:10FE90006E7466006170702073746172740D0A0074
:10FEA0006E756D6265723A256420200076616C691A
:10FEB000643A25642000000070726F746F636C3ABE
:10FEC0002564200052533438352054583A0000003D
:10FED000C046C046C046C046FFF74AFE6164646C37
:10FEE000697374007365746D706F77006765746D06
:10FEF000706F770073696D756C7478007265626FEE
:10FF00006F740000252E32780000000049444C45F3
:10FF100000000000546D722053766300546D7251DE
:10FF200000000000706C632052583A0034383520CD
:10FF300052583A007665720008000000F0E300E0D5
:10FF4000EEEEEEEEFFF7FEBFFFF7FEBFFFF7FEBFE0
:10FF5000FFF7FEBFFFF7FEBFFEF719B9FFF7FEBFC1
:10FF6000FEF7F2B8FBF766BDFFF7FEBFFFF7FEBF77
:10FF7000FFF7FEBFFFF7FEBFFFF7FEBFFEF7AEB90C
:10FF8000FFF7FEBFFFF7FEBFFFF7FEBFFFF7FEBFA5
:10FF9000FFF7FEBFFFF7FEBFF7F78ABBFFF7FEBF15
:10FFA000F5F7C6B8FFF7FEBFFFF7FEBFF5F7E8B8F5
:10FFB000FFF7FEBFFFF7FEBFFFF7FEBFFFF7FEBF75
:10FFC000FFF7FEBFFFF7FEBFFFF7FEBFFFF7FEBF65
:10FFD000FFF7FEBFFFF7FEBFFFF7FEBFFFF7FEBF55
:10FFE000FFF7FEBFFFF7FEBFFFF7FEBFFFF7FEBF45
:10FFF000FFF7FEBFFFF7FEBFFFF7FEBFF5F7B2B892
:020000040801F1
:10000000F5F7D8B8F7F77CBBFFF7FEBFFFF7FEBFE9
:10001000FFF7FEBFFFF7FEBFFFF7FEBFFFF7FEBF14
:10002000FFF7FEBFFFF7FEBFFFF7FEBFFFF7FEBF04
:10003000FFF7FEBFFFF7FEBFF5F7E4B8F5F728B905
:10004000FFF7FEBFFFF7FEBFFFF7FEBFFFF7FEBFE4
:10005000FFF7FEBFF5F7BCB8200600C1814001C024
:10006000804104610C2108E118A11CF10B30F1075B
:1000700038F12760F11F70F1206000FEC0C101C39C
:100080000302C2C60607C705C5C404CC0C0DCD0FBC
:10009000CFCE0E0ACACB0BC90908C8D81819D91B6C
:1000A000DBDA1A1EDEDF1FDD1D1CDC14D4D515D7EC
:1000B0001716D6D21213D311D1D010F03031F1333C
:1000C000F3F23236F6F737F53534F43CFCFD3DFFFC
:1000D0003F3EFEFA3A3BFB39F9F83828E8E929EBCC
:1000E0002B2AEAEE2E2FEF2DEDEC2CE42425E5272C
:1000F000E7E62622E2E323E12120E0A06061A1639C
:10010000A3A26266A6A767A56564A46CACAD6DAF3B
:100110006F6EAEAA6A6BAB69A9A86878B8B979BBEB
:100120007B7ABABE7E7FBF7DBDBC7CB47475B5776B
:10013000B7B67672B2B373B17170B05090915193FB
:1001400053529296565797559594549C5C5D9D5F7B
:100150009F9E5E5A9A9B5B99595898884849894B4B
:100160008B8A4A4E8E8F4F8D4D4C8C4484854587AB
:100170004746868242438341818040001101F375E6
:100180000100016220091003480040802508121078
:100190000453040C153204032003000C0140080F23
:1001A00082080C21C043270C3810031C00024004B5
:1001B0000812FF0F83F877538200464102F301389B
:1001C0000164250E22025C60010140042D510C21C6
:1001D0006443250E3822446443380164C0037A0026
:1001E00020F87B687550D0034400406009644300E8
:1001F00002845158C30800644326113822806411D8
:1002000008226464C0037C0020508464620209F206
:10021000034C644208BC5002100140100F610C21D5
:100220003843343B3813580464564C2C127DC8C2F2
:100230007E64620809F2035064421010515831D4B0
:1002400060011401404152353861433164127F64CA
:10025000C28064F33180000120020102030404A083
:100260000206070809142110838000A492400C9311
:1002700000020C92010C8B80006482400C32AA01B7
:1002800030010000990130010000110141184010B7
:10029000020406080090D00300FF010001010605DA
:0D02A000A485E40006901F1F9008000D01CA
:040000050800FED120
:00000001FF
